:100000000C9423050C945B050C945B050C945B0528
:100010000C945B050C945B050C945B050C945B05E0
:100020000C945B050C945B050C94F4170C94CD1D9B
:100030000C94FF280C945B050C945B050C945B05F9
:100040000C945B050C945B050C945B050C945B05B0
:100050000C945B050C94CD180C945B050C945B051B
:100060000C945B050C945B050C945B050C945B0590
:100070000C945B050C945B050C945B050C945B0580
:100080000C945B050C945B050C945B050C945B0570
:100090000C945B050C945B050C945B050C945B0560
:1000A0000C945B050C945B050C945B05050109023F
:1000B000A10185020901A100050919012905150001
:1000C00025019505750181029501750381010501E1
:1000D000093009311581257F950275088106093897
:1000E0001581257F950175088106050C0A380215D2
:1000F00081257F950175088106C0C005010980A191
:1001000001850319012AB700150126B7009501756D
:10011000108100C0050C0901A101850419012AA064
:1001200002150126A002950175108100C005010984
:1001300006A1018506050719E029E71500250195A7
:1001400008750181020507190029EF1500250195A1
:10015000F0750181020508190129059505750191C0
:1001600002950175039101C00660FF0961A10109B3
:1001700062150026FF0095207508810209631500AD
:1001800026FF00952075089102C005010906A1010E
:10019000050719E029E71500250195087501810279
:1001A0009501750881010507190029FF150026FF33
:1001B0000095067508810005081901290595057542
:1001C000019102950175039101C00000000000003B
:1001D000000000000000000000000000000000001F
:1001E00000000000000000000000000000007E0F82
:1001F00000D4FFFFFFC700000078000000000000EF
:1002000000002A2B28000000000000000000000071
:10021000000000000029000000002C1E34202122D4
:1002200024342627252E362D3738271E1F2021223D
:10023000232425263333362E37381F0405060708B6
:10024000090A0B0C0D0E0F101112131415161718A6
:10025000191A1B1C1D2F3130232D350405060708E4
:10026000090A0B0C0D0E0F10111213141516171886
:10027000191A1B1C1D2F3130354CFD377A585A0086
:100280000004E6D6B4460200210116000000742FD7
:10029000E5A3E00433016C5D003D8889C65436C394
:1002A000174FE4E17AD4E4CBBA20C2C2A5DD57AD42
:1002B000ED82AE5352EE6D1E08C47EEC844BA14A13
:1002C000FA3FDC0273341D78ED78CB714453218AF8
:1002D000E63DD180D584EFD94B940CA408D09ACCBC
:1002E00085E8EE3919FACF346B2A63901081157EB8
:1002F000F0128FB5004516771169DDCCEE6A84E403
:1003000066243818E6E3C40136B328D2EF7CC7F17F
:10031000FF6C41A6070298D5D5D2D24BB2DF52C6A8
:10032000745B6796D313D5744C1837958FE0905152
:1003300021916D603949947341CA9E05ABFDA6C5F4
:100340002050F22C35C8CE93C648292DAD6E98208A
:10035000779FA515D9A096200B055A7D5893B50C0B
:10036000A72C3E521DED94827880EAD002FCDA4739
:10037000EF9FB8C67CDF8AEB9D9D88807D0FDC25D2
:100380005AAEF6C60B368D244CBE818090AE7EDC14
:10039000027611DE407742AC268C5BF32DDD5A9C51
:1003A0000E02ACCD6F28EACB1E7FA7B91291F3DF06
:1003B0008DCC2390B03B5DB521DA81A3D4822899FE
:1003C000EF7FD4EE6CF3AA7C8FB8C8DB98F92831A4
:1003D000DC1C3B2918EF8E1503474C84DF17D1EA4C
:1003E0008269E893EDC2B4F372BAD91E0EDB6B9347
:1003F0003C6CDC4F06ACA8563ADBF3DAA12CA4DD4A
:10040000989D2BBEEB00C98F099CE01ACBF400012C
:100410008803B4080000CDB015EAB1C467FB020040
:1004200000000004595A000000000200010006000C
:1004300002000C0003000D0004000E0005000F0078
:10044000060011000700130008001400090017003F
:100450000A0018000B001F000C0020000D002100F6
:100460000E0023000F00270010002A0011000001D9
:100470000101010101010101020202020202020264
:100480000203030303030303030404040404040436
:1004900005050505050606060606070707070708FA
:1004A000080808090909090A0A0A0B0B0B0C0C0CAD
:1004B0000D0D0D0E0E0E0F0F0F1010111111121247
:1004C00013131414151516161717181819191A1AC4
:1004D0001B1B1C1D1D1E1E1F202021222223242425
:1004E000252626272829292A2B2C2D2D2E2F303161
:1004F0003232333435363738393A3B3C3D3E3F4073
:100500004142434445464748494A4C4D4E4F50515D
:100510005354555658595A5B5D5E5F616264656617
:1005200068696B6C6D6F7072737577787A7B7D7E9E
:100530008082838587888A8C8E8F91939596989AEE
:100540009C9EA0A2A3A5A7A9ABADAFB1B3B5B7BA06
:10055000BCBEC0C2C4C6C9CBCDCFD1D4D6D8DBDDDA
:10056000DFE2E4E7E9EBEEF0F3F5F8FAFDFF002651
:100570003646002737470028384800293949002ADD
:100580003A4A002B3B4B01263646012737470128C4
:10059000384801293949012A3A4A012B3B4B0226A6
:1005A00036460227374702283848007464540075DD
:1005B00065550076665600796959007A6A5A007B5B
:1005C0006B5B017565550176665601796959017A4B
:1005D0006A5A017B6B5B027464540275655502763E
:1005E000665600A4948400A5958500A6968600A76B
:1005F000978700A8988800A99989027B6B5B01A462
:10060000948401A5958501A6968601A7978701A8E0
:10061000988801A9998902796959027A6A5A002E43
:100620003E4E002F3F4F00304050003141510032CC
:1006300042520033435301AC9C8C012E3E4E012F9D
:100640003F4F01304050013141510132425201339C
:10065000435302A7978702A89888007C6C5C007DB2
:100660006D5D007E6E5E008171610082726200834A
:10067000736301AD9D8D017C6C5C017D6D5D017EC0
:100680006E5E01817161018272620183736302A9EE
:10069000998900AC9C8C00AD9D8D00AE9E8E00AF04
:1006A0009F8F00B0A09000B1A19101AE9E8E01AFCE
:1006B0009F8F01B0A09001B1A19102293949022A6E
:1006C0003A4A022B3B4B29003A003B003C003D00DC
:1006D0003E003F004000410042004300440045000E
:1006E0004C00460035001E001F00200021002200A3
:1006F0000000230024002500260027002D002E00E6
:100700002A002B0014001A000800150017004B00E7
:100710001C0018000C00120013002F0030003100E4
:10072000390004001600070009000A002A000B0027
:100730000D000E000F003300340028004E00E100D1
:100740001D001B0006001900050028001100100004
:10075000360037003800E50052000000E000E300FA
:10076000E20000002C00E000E1002C000000E600A8
:100770000151E400500051004F00005C01000100F5
:10078000010001000100010001000100B200B300FE
:10079000AF00B100145CDE5C01000100010001004B
:1007A0000100010000000100010001000100010042
:1007B000010001005300C25CC35CC95CC55C010060
:1007C00001004A00010001000100010001000100D8
:1007D000010001000100CC5CCA5CCB5C010001009F
:1007E0000100010001000100010001000100010001
:1007F0004D000100010001000100010001000100A5
:1008000001000100010001000100A800A900000092
:1008100001000100010000000100010001000100D1
:10082000000001000100AE00AC00AA00AB00010016
:1008300001000100010001000100010001000100B0
:1008400001000100010001000100010001000100A0
:100850000100010001000100000001000100010091
:100860000100010001000100010001000100010080
:100870000100010001000100010001000100010070
:100880000100010001000100010001000100010060
:100890000100010001000100010001000100010050
:1008A0000100010001000100010001000100010040
:1008B0000100010001000100010001000100010030
:1008C0000100000001000100010000000100010022
:1008D0000100010000000100010001000100010011
:1008E0000100010001000100010001000100010000
:1008F00001000100010001000100010001000100F0
:1009000001000100010001000100010000000100E0
:1009100001000100010001000100010001000100CF
:1009200001000100010001000100010001000100BF
:1009300001000100010001000100010001000100AF
:10094000010001000100010001000100010001009F
:10095000010001000100010001000100010001008F
:10096000010001000100010001000100010001007F
:100970000100010001000000010001000100000071
:100980000100010001000100000001000100010060
:1009900001000100010009025B00030100A0FA0947
:1009A000040000010301010009211101000122409E
:1009B000000705810308000109040100020300008B
:1009C00000092111010001222200070582032000F5
:1009D00001070503032000010904020001030000D0
:1009E0000009211101000122BC0007058403200039
:1009F00001120100020000000842586E4B01000184
:100A00000203011C037600690061006C003A006675
:100A100000360034006300320062003300630000DF
:100A2000000E034B004E00490047004800540000F0
:100A3000000E0358002D0042004F005700530000E5
:100A400000040309040011241FBECFEFDAE0DEBF6B
:100A5000CDBF04B603FE18C080916A0690916B0664
:100A6000A0916C06B0916D068730904BA740B04BBB
:100A700059F410926A0610926B0610926C0610924E
:100A80006D06E0E0F8E3099526E0ACEDB2E001C0C8
:100A90001D92AA36B207E1F712E0A0E0B1E0EEEA5B
:100AA000F5E602C005900D92AC3DB107D9F70E9462
:100AB00026290C949F320C940000E8EDF0E0808130
:100AC0008E7F80831092E2001092DA001092E10093
:100AD000A0EEB0E08C9181608C9380818F778083D1
:100AE00019BCA7EDB0E08C918E7F8C9380818F7EB6
:100AF00080831092040608952091E4003091E5006F
:100B000095E6A9012091EC00822F817020FF06C09C
:100B10008091E80080FF06C080E008952091E80001
:100B200022FD1AC080913206882389F0853089F031
:100B30008091EB0085FD0FC02091E4003091E5002D
:100B400042175307F9F29150E1F684E0089582E0EC
:100B5000089583E0089581E00895EF92FF920F9346
:100B60001F93CF937C018B010E947C05C82F8111BC
:100B700017C08091E80085FD0BC08091E8008E775A
:100B80008093E8000E947C05882399F3C82F08C051
:100B9000F70181917F018093F1000150110949F71C
:100BA0008C2FCF911F910F91FF90EF900895CF93CD
:100BB000FC0180913206843001F5C091E900CF70CC
:100BC0002091EC00922F917020FD90E8C92B82E0DB
:100BD0008093E9008091E80080FF0CC050E040E085
:100BE00060E270E0CF010E94AD058091E8008E7751
:100BF0008093E800CF70C093E900CF910895809171
:100C00002A0687FF13C08091E80082FF06C080910A
:100C1000E8008B778093E80004C080913206811150
:100C2000F2CF0895809132068823D9F38091E800AD
:100C300080FFF8CF8091E8008E77ECCF982F9093CB
:100C4000E900242F762F50E0891731F07091EC00E5
:100C50002091ED005091F00021FD07C09F5F97307B
:100C600071F78093E90081E008953091EB003E7FB9
:100C70003093EB003091ED003D7F3093ED003091EB
:100C8000EB0031603093EB007093EC002093ED00AB
:100C90005093F0002091EE0027FDE0CF80E0089512
:100CA000B0E0A0E0E6E5F6E00C94FE30C8EDD0E060
:100CB00088818F7E8883E7EDF0E08081816080838A
:100CC00084E082BF81E08093040688818E7F8883E0
:100CD00002EE10E0F80110821092DA0081EEC82EC8
:100CE000D12CF601108288818F7788838881806873
:100CF000888388818F7D888319BC10923206109278
:100D00002906109228061092270690EEE92EF12C63
:100D1000F70180818B7F808388818160888342E0B6
:100D200060E080E00E941E06F60180818E7F808355
:100D3000F801808181608083808188608083F701F1
:100D400080818E7F8083888180618883CDB7DEB784
:100D5000E8E00C941A31FC01809130069091310644
:100D600086179707A0F06115710529F49091E800A6
:100D70009E779093E80090E06115710551F4911110
:100D800008C08091E80082FF34C080E00895BC0173
:100D9000F2CF809132068823C1F18530C1F1809174
:100DA000E80083FD30C08091E80082FDEACF8091A9
:100DB000E80080FFE1CF8091F3002091F200382F0E
:100DC0006115710519F02830310558F091E028308F
:100DD000310509F090E02091E8002E772093E8009B
:100DE000CBCF81918093F100615071092F5F3F4F0C
:100DF000E7CF80913206882341F0853041F0809121
:100E0000E80083FFBECF81E0089582E0089583E08B
:100E100008950895809106060895209113012223D4
:100E2000C9F02091FF0527FF15C0E62FE695E6954E
:100E3000E695EE31D8F4E80FF92FF11D677021E047
:100E400030E001C0220F6A95EAF7209582812823BD
:100E500022830895FC01329608962191621303C003
:100E6000DF0111971C92E817F907B9F7089520914F
:100E700013012223C1F02091FF0527FF14C0E62FA4
:100E8000E695E695E695EE31F8F4E80FF92FF11DB9
:100E9000677021E030E001C0220F6A95EAF7828195
:100EA000822B82830895FC0132962FEF30E041912E
:100EB000641751F02F3F19F4411101C0232F3F5FF8
:100EC0003630A9F72F3F09F40895820F911D27FDB1
:100ED0009A95FC01628308952091F8053091F905F7
:100EE0002817390771F09093F9058093F805E09180
:100EF000F605F091F705309721F00084F185E02D9B
:100F0000099508952091F4053091F50528173907C2
:100F100071F09093F5058093F405E091F605F0915A
:100F2000F705309721F00680F781E02D09950895A7
:100F3000E091F605F091F705309729F00190F081E6
:100F4000E02D0995089580E00895FA01811101C00E
:100F5000FB0109950895E7E3F6E0248130E1231BC6
:100F600008F420E024838091ED0381608093ED03F9
:100F70000895E7E3F6E0248130E1230F08F42FEF32
:100F800024838091ED0381608093ED030895909117
:100F90003706937071F08093380660933906493CA8
:100FA00008F048EC40933A068091ED03822B809341
:100FB000ED030895E7E3F6E0438120E1421B08F4E6
:100FC00040E0818121E0628190E00E94C70708959E
:100FD000E7E3F6E0438120E1420F08F44FEF81811F
:100FE00021E0628190E00E94C7070895E7E3F6E000
:100FF000628120E1621B08F460E0818121E043818D
:1010000090E00E94C7070895E7E3F6E0628120E1DF
:10101000620F08F46FEF818121E0438190E00E942C
:10102000C7070895E7E3F6E0818121E0438162810B
:101030008850990B0E94C7070895E7E3F6E0818185
:1010400090E021E04381628108960E94C7070895DD
:1010500090913706937061F081110BC0946090936A
:101060003706109212018091ED03862B8093ED03D9
:101070000895823110F09464F2CF880F880F982B76
:10108000EECF8091370686958695815009F481E1EF
:1010900061E00E942808089580913706869586951C
:1010A0008F5F823108F081E061E00E942808089596
:1010B000EF92FF920F939701201B31092F3F3105CB
:1010C00019F010F02FEF30E02095382F320F08F490
:1010D0003FEF832F0F91FF90EF900895EF92FF92D3
:1010E0000F939701201B31092F3F310519F010F0A4
:1010F0002FEF30E0322F3095482F430F08F44FEF99
:10110000842F620F0F91FF90EF900895EF92FF925E
:101110000F931F930E0D1F2D111DF90137FF03C0F3
:10112000F195E195F10924E0EE0FFF1F2A95E1F713
:10113000EF3FF10519F014F0EFEFF0E09A0157FFDF
:1011400003C031952195310994E0220F331F9A9500
:10115000E1F72E173F070CF4F901E00FF11FEF3F05
:10116000F10519F010F0EFEFF0E0E095282F3E2F99
:10117000230F08F42FEF822F1F910F91FF90EF9014
:101180000895EF92FF920F93970195E0099F200D2C
:10119000311D11242F3F310519F010F02FEF30E0F1
:1011A0002095382F320F08F43FEF832F0F91FF90D7
:1011B000EF90089522E8241B08F420E0620F0895C0
:1011C0004095282F429F412D1124842F0895EF929E
:1011D0000F93972F23E0029FB00111247595679517
:1011E0006E0D792F0F91EF900895E42FF0E0EE0F40
:1011F000FF1FE652FE4F6081621B0895E42FF0E06E
:10120000EE0FFF1FE752FE4F6081621B0895622FB1
:1012100008950E94A41308950E94661308950F93E1
:101220001F9310E0F801EE0FFF1FE752FE4F908171
:101230009C5597FD9195000F111FF801E652FE4F46
:1012400000810152110B2003F001219FF00D1124A8
:1012500008E310E0091B110997FD13954003900165
:10126000419F300D1124E20FF31F9F01220F331F06
:101270002E0F3F1F37FF02C021583F4F220F232F51
:10128000221F330B620F1F910F910895FC019B01E8
:10129000009729F480E077FF2BC080E80895AC0127
:1012A00097FF04C044275527481B590BB901640F09
:1012B000751F37FD10C0241B350BC901A5E0880F31
:1012C000991FAA95E1F70E942B3180E2861BF7FF58
:1012D0000FC081950895CB0165E0880F991F6A952D
:1012E000E1F7BA01621B730B0E942B3180E6EECF4F
:1012F0000895EF920F93CF93DF93D72FC82FC90193
:101300000E19BA010E944609602F681B7D2F8C2F91
:10131000DF91CF910F91EF900895EF920F931F936C
:10132000CF93DF93D62FC72F182FC9010E19010FA6
:10133000BA010E944609081B202F219F212D11244C
:10134000822F6D2F7C2FDF91CF911F910F91EF9006
:1013500008950F93CF93DF93D72FC82FC901BA01F8
:101360000E944609682F600F7D2F8C2FDF91CF914F
:101370000F910895E82F86FDE0952E2F2F7086FDA2
:101380002F5FE695E695E695E670F0E0E859FE4FAA
:101390009181929F902D212D112492959F702295DD
:1013A000207F922B2081920F87FD919580E8890FF5
:1013B0000895AC018230910508F408959FEF413EF5
:1013C0008EE1580740F49A0195E0369527959A9555
:1013D000E1F798E0920F61E0E62FE90FFF27FF1F8A
:1013E0009F0135952795822F229FF001239FF00DB5
:1013F000F00D11244E175F0738F49FEF920F9617E8
:1014000058F78FEF860F08952F3FE9F361E0620FE1
:10141000F6CF30E020E0869F212D969F200D311DD4
:101420001124C9010895AF92BF92CF92DF92FF922B
:101430000F931F93CF93DF93362F472FE82FF0E0C2
:10144000E259FB4F71110FC0E4918E2F2E2F6E2F9A
:10145000722FDF91CF911F910F91FF90DF90CF906E
:10146000BF90AF900895C72FD0E02491F22E022FA5
:1014700010E056E0659FC0011124EFEFF0E0BF01DE
:101480000E94E030832F90E0880F991F35E5369F4A
:10149000D001379FB00D11248A1B9B0B982F990FF9
:1014A000980F6F01CC1ADD0AC09ED001C19EB00D0D
:1014B000D09EB00D11248B2F499FA0011124452FE0
:1014C00055276F01C41AD50AC09EA001C19E500DB8
:1014D000D09E500D11245F01A91AB108AC9E600185
:1014E000AD9ED00CBC9ED00C1124CD2CDD24EC196B
:1014F000FD09E09FE001E19FD00DF09FD00D112488
:10150000ED2F62307105A1F050F46115710509F4F9
:101510009ECF6130710581F0EB2F852F98CF64301D
:10152000710569F080F06630710509F490CFF4CF51
:10153000E22F2B2F8D2F8BCFE22F252F88CFEB2F54
:10154000822F2D2F84CF2B2F8F2DE52F80CF2F9201
:101550003F925F926F927F928F929F92AF92BF92D3
:10156000CF92DF92EF92FF920F931F93CF93DF936F
:10157000CDB7DEB72A970FB6F894DEBF0FBECDBF4A
:101580008B837E836D832091140182E1289F802DBF
:1015900011248F838E5E89838A83873510F036E528
:1015A0003A8380913D068C83FF81EF2FF0E0FA872C
:1015B000E987CF01880F991F9C0127523E4F69018F
:1015C0003B81832F90E0FC013196F887EF838A817D
:1015D00099859817E8F081E0E981E63508F080E028
:1015E0002A960FB6F894DEBF0FBECDBFDF91CF9124
:1015F0001F910F91FF90EF90DF90CF90BF90AF9031
:101600009F908F907F906F905F903F902F90089564
:10161000E985FA85EB57FD4F80819091150189236B
:10162000F1F020903806309039062F813885235C00
:10163000394F39015B8010E0FC815F16D0F02091BA
:101640003A06129F112D1124B101812F0E94130A15
:10165000462F282F672F89859A850E940C09298596
:101660003A852F5F3F4F3A87298732E0C30ED11C5E
:10167000AECFF30181913F01F601A080A81ABB080B
:101680008180F3018781881A9908AA9C9001AB9CFC
:10169000300D300D1124889CC001899C900D900D57
:1016A0001124820F931F0E94D909082F60913B06D5
:1016B00021E0620F08F46FEFF301EE0FFF1FED530F
:1016C000F640858996890E94090A7C019401A5014A
:1016D000B101812FED81FE8109951B015394182FD3
:1016E000ABCFB0E0A0E0E7E7FBE00C94FE308C016C
:1016F000C091140182E1C89FC02D112422E1D22E95
:10170000DC0ECD2C26E52D1510F496E5C92E209182
:101710003B0631E0230F08F42FEF30E050E040E0CB
:101720006FEF7FEF80E090E00E943C327901D0E0E3
:101730002C2FCC1550F081E0F5E5FD1508F480E084
:10174000CDB7DEB7E8E00C941A31FE01EB57FD4F40
:10175000808190911501892311F140913D064150FE
:10176000042E000C550B47FF1CC0C70160913B06BF
:1017700021E0620F08F46FEF0E94090AAC0160914A
:1017800038067091390680913A06F80109950E9451
:10179000130A462F282F672FCE010E940C0921968D
:1017A000C7CFFA01E35CF94F818982130AC0FA01BD
:1017B000EE0FFF1FE35CF94F818D928D8E159F0513
:1017C000A8F241505109CFCFB0E0A0E0EAEEFBE033
:1017D0000C94F9305C01C091140182E1C89FC02DC6
:1017E000112412E11C0FF12E173510F036E5F32EFF
:1017F00060913B06669580913306909134060E9475
:10180000090A782ED0E0CF1548F081E0163508F0AF
:1018100080E0CDB7DEB7EDE00C941531FE01EB575B
:10182000FD4F8081909115018923C9F1CE01880F68
:10183000991F81589E4FFC01E65AFF4F2081422F8D
:101840004C55550B6A01855A9F4FFC018081282F0A
:101850002152330B4901449F9001459F300D300DBB
:101860001124889CC001899C900D900D1124820F39
:10187000931F0E94D909082F60913806709139068C
:1018800080913A06E72C9401A601F50109950E9482
:10189000130A462F282F672FCE010E940C0921968C
:1018A000B2CFB0E0A0E0E7E5FCE00C94FF307C01B3
:1018B000C091140182E1C89FC02D112412E11C0FB8
:1018C000012F173508F006E560913B066695669591
:1018D00021E0620F08F46FEF809133069091340697
:1018E0000E94090AD82ED0E0C01748F081E01635D2
:1018F00008F080E0CDB7DEB7E7E00C941B31FE01C5
:10190000EB57FD4F808190911501892391F06091F3
:1019100038067091390680913A062D2D4C2FF7012B
:1019200009950E94130A462F282F672FCE010E9487
:101930000C092196D9CF9091BB03803F59F4809137
:10194000BC0387FF0DC01092BC0391110BC0109215
:10195000B30308C0813F81F48091BC0318169CF347
:10196000992381F08091BD039091BE03892B09F0EA
:1019700064C01092B2030895823F49F497FFF0CFFC
:101980001092BB038091BC038111ECCFE0CF833F69
:1019900019F41916ACF3E4CF2091BD03893F29F463
:1019A0001216F4F61092BD03DBCF8A3F19F427FF1D
:1019B000D7CFF8CF2091BE038B3F29F427FFD0CF9C
:1019C0001092BE03CDCF8C3F19F41216CCF3C8CFC2
:1019D000843F31F48091BA038E7F8093BA03C0CFE5
:1019E000853F21F48091BA038D7FF7CF863F21F4A4
:1019F0008091BA038B7FF1CF873F21F48091BA03A6
:101A0000877FEBCF883F21F48091BA038F7EE5CFAB
:101A10008D3F31F48091B4038E7F8093B403A0CFC7
:101A20008E3F21F48091B4038D7FF7CF8F3F09F073
:101A300097CF8091B4038B7FF0CF08958091B4034A
:101A400080FD16C081FD16C082FD16C08091B203D4
:101A50008823A1F0883280F428E0829FC0011124FD
:101A600068E270E00E942B31862F672B39F00895D1
:101A700082E0089584E0089588E0089581E0089563
:101A80008091B40380FD14C081FD14C082FD16C096
:101A90008091B303882381F08E3180F420E5829F0A
:101AA000C00111246EE170E00E942B31862F089551
:101AB00084E1089588E2089588E0089580E5089516
:101AC000803F31F40E94400D81958093BC030895BE
:101AD000813F19F40E94400DF8CF823F31F40E94FB
:101AE000400D81958093BB030895833F19F40E94B4
:101AF000400DF8CF893F29F40E941E0D8093BD034D
:101B000008958A3F21F40E941E0D8195F7CF8B3FE7
:101B100031F40E941E0D81958093BE0308958C3F81
:101B200019F40E941E0DF8CF843F31F48091BA035E
:101B300081608093BA030895853F21F48091BA03B0
:101B40008260F7CF863F21F48091BA038460F1CFA1
:101B5000873F21F48091BA038860EBCF883F21F45E
:101B60008091BA038061E5CF8D3F31F48091B40359
:101B700081608093B40308958E3F21F48091B40373
:101B80008260F7CF8F3FB9F78091B4038460F1CFC3
:101B900080E00895F894E82FE295EF70F0E031A12D
:101BA000282F2F7081E090E001C0880F2A95EAF776
:101BB000982F9095932391A392A1892B82A3789437
:101BC00008959091FF0592FF06C0282F28712830B4
:101BD000F9F4877F846093FF06C0282F287128318D
:101BE000F1F4877E84612091000620FF06C0382F23
:101BF00038713830D9F4877F816021FF06C0282FE3
:101C000028712831D1F4877E816194FD877E089503
:101C1000282F24712430F9F68B7F8860DCCF282FA1
:101C20002471243101F78B7E8861DDCF382F31712B
:101C3000313019F78E7F8860E0CF282F2171213154
:101C400021F78E7E8861E1CFCF93DF93EC0182385C
:101C50009105A9F1D8F58133910509F496C048F5AD
:101C60008932910509F48AC08A9709F495C0C11593
:101C700021E5D20708F0BCC0C11530E5D30708F054
:101C800014C1C83ED10508F09CC0C03ED10560F526
:101C9000C83AD10508F087C0C53AD10508F0FDC0A3
:101CA000C130D10509F12097F9F0C430D105E0F435
:101CB00040C08533910509F45AC0C997C1F6809197
:101CC000FF05837089F0C0EED0E00EC0833E910521
:101CD00099F170F4803E910501F1823E910539F64B
:101CE0008091FF0582FD21C0CE01DF91CF91089543
:101CF000863E910561F1873E910571F1843E910523
:101D000009F0B5CF8091000681FFEECF8091FF05ED
:101D1000C7EED0E084FD0DC0E7CF8091FF0580FDC8
:101D200012C19091000690FFDFCFC3EED0E084FF98
:101D3000DBCFD0E0C0E0D8CF8091FF0582FD06C1A7
:101D40009091000690FDBFCF84FFCECFF2CF80915F
:101D5000FF0583FDDDCFC8CF8091FF0583FDF9C06E
:101D60009091000691FFF0CFC4EED0E0BDCF8091FE
:101D7000FF0585FFB9CFC9E2D0E0B6CF8091FF055E
:101D800085FFB2CFC5E3D0E0AFCF8091FF0586FFDE
:101D9000ABCFCAE2D0E0A8CF8091FF0586FFA4CFE9
:101DA000C1E3D0E0A1CFCF3BD10518F6C85AD0E0AF
:101DB000CC0FDD1FCB5DDE4F0990D881C02DD464E0
:101DC00093CFC11540E2D40758F4C11581E0D8077C
:101DD00008F08ACFC03FD10508F4ABCFD06584CFDF
:101DE000C11590E4D90708F4A4CFDF70D06A7CCF86
:101DF000C11525E5D20700F5C11534E5D30708F074
:101E00008AC0C11543E5D40708F071C0C11582E549
:101E1000D80708F467C0CE018370992721E030E02D
:101E200002C0220F331F8A95E2F7C695C69580E25D
:101E3000C89FE001112452C0C11599E5D907A8F443
:101E4000C11528E5D20708F06BC0C11536E5D307E8
:101E500008F06FCF8C2F0E94E10DC82FD0E0DC2F4F
:101E6000CC27CC27DF71D0623FCFC1154AE5D4071C
:101E700008F45BC0CE0190568115904208F059CF0E
:101E80008D2F8F710E94E10D90E0982F8827882771
:101E90009F719C012C2BE901E6CFC55AD0E0CE5DA5
:101EA000DE4FC881D0E0D0641FCFCE01E4E096952C
:101EB0008795EA95E1F783702C2F26952695237058
:101EC00040E2249F90011124382B8C2F8370C1E0B5
:101ED000D0E002C0CC0FDD1F8A95E2F7C22BD32BD6
:101EE000DC6802CFDC2FCC27C16FD06AFDCECE01DB
:101EF0008370992721E030E002C0220F331F8A95BA
:101F0000E2F7C695C69590E2C99FE0011124C22B65
:101F1000D32BDA68E9CEDC2FCC27C46FD06AE4CEAD
:101F2000DC2FCC27C06FD06ADFCE8C2F8F700E9441
:101F3000E10D34E0D695C7953A95E1F7CF709C2F27
:101F4000EC01D069D1CEC9E3D0E0CECEC2EED0E074
:101F5000CBCEC6EED0E0C8CE80918303882331F08B
:101F6000109283031092820310928103089580954A
:101F700090918003982390938003089510925E03BC
:101F800010925D0310925C03089580915B03909121
:101F90002A03981301C008958F5F8770FACF292F05
:101FA000963078F58F3068F590E03FE0239F800D04
:101FB000911D1124682F677023E0969587952A95C7
:101FC000E1F7FC01EE0FFF1FE80FF91FE050FD4F96
:101FD00050E040E080E0219130E0062E02C03695CE
:101FE00027950A94E2F721703327042E01C0220FAF
:101FF0000A94EAF7822B4F5F5F4F4330510559F740
:10200000089580E00895292F963098F58F3088F54F
:1020100090E03FE0239F800D911D1124282F277011
:1020200041E001C0440F2A95EAF723E09695879591
:102030002A95E1F7FC01EE0FFF1FE80FF91FE050B2
:10204000FD4F30E020E070E05191DF011197CB01AE
:10205000022E02C0969587950A94E2F781708195C9
:102060008527842385278C932F5F3F4F23303105AD
:1020700059F708959C013A9521153F4150F5FC010F
:10208000EE27F170BC0166277270AC0144275470D2
:102090009C012227387094FF0EC080E1EF2B09F4D9
:1020A00080E0672B09F08062452B09F08064232BC8
:1020B00089F08068089581E0EF2B09F480E0672BB8
:1020C00009F08260452B09F08460232B19F08860A9
:1020D000089580E00895809301067093030660934D
:1020E0000206809132068430F9F48093E9008FEF84
:1020F0009091E800815095FD06C095ED9A95F1F715
:1021000000008111F5CF8091E80085FF0DC050E0FF
:1021100040E063E070E081E096E00E94AD058091D0
:10212000E8008E778093E8000895BC0184E00E9467
:102130006B100895BC0183E00E946B1008959C0110
:1021400084E08093E9009FEF8091E800915085FD45
:1021500006C085ED8A95F1F700009111F5CF8091C9
:10216000E80085FF0CC050E040E066E070E0C90187
:102170000E94AD058091E8008E778093E800089575
:10218000CF93DF93EC01809113018823B1F180910B
:10219000FF0587FF32C060E284E08093E9008FEFA3
:1021A0009091E800815095FD06C095ED9A95F1F764
:1021B00000008111F5CF8091E80085FF1BC0809160
:1021C000130170E050E040E0811104C050E040E0B5
:1021D00068E070E0CE010E94AD058091E8008E7746
:1021E0008093E80080E2FE01A7E0B6E001900D9246
:1021F0008A95E1F7DF91CF91089568E081E0CDCF36
:1022000081E08093E00080E28093D8001092C900C2
:102210008FE19EE40197F1F700C0000087E090EBAA
:10222000DC0180936A0690936B06A0936C06B093D2
:102230006D0688E19CE00FB6F894A8958093600045
:102240000FBE90936000FFCFCF93DF93C7EFD2E034
:1022500060E0CE010E9418322196C11584E0D807B3
:10226000B9F7DF91CF9108951F93CF93DF93122F8A
:102270008430E0F46630D0F44F30C0F4C42FD0E0A6
:10228000CC0FDD1F9EE1699FC00DD11D112494EB81
:10229000899FC00DD11D1124632FCE0187960E9406
:1022A0001832612FCE0188960E941832DF91CF91AB
:1022B0001F9108958F929F92AF92BF92CF92DF921B
:1022C000EF92FF921F93CF93DF938090EE05909053
:1022D000EF0581E090E09093EF058093EE0586ECAA
:1022E000C82E86E0D82ED0E07601C0E014C0F501FB
:1022F00025913491412F6C2F8D2F0E94341182E053
:10230000A80EB11C1F5F1F3091F78EE1E80EF11C83
:10231000CF5FC63019F0570110E0E9CFDF5F84EBE3
:10232000C80ED11CD43001F79092EF058092EE05D3
:10233000DF91CF911F91FF90EF90DF90CF90BF90F2
:10234000AF909F908F900895CF93C82F6FEF81111A
:102350006CE283E290E00E9418326FEFC11162ECF0
:1023600084E290E00E9418326FEFC1116EEB85E2BB
:1023700090E00E941832CF91089580E00E94A4114D
:1023800060E086E290E00E9418320E945A110E949A
:10239000241181E00E94A41108950F931F93CF93FD
:1023A000DF93843030F5663020F54F3010F5C42FC0
:1023B000D0E0CC0FDD1F2EE1629FC00DD11D112496
:1023C00034EB839FC00DD11D1124CE0187960E944E
:1023D000FA31082F10E0102F0027CE0188960E94B6
:1023E000FA319801282BC901DF91CF911F910F91EC
:1023F000089590E080E0F8CF462F2091F2053091CB
:10240000F305232B99F4703F39F4603F79F4809100
:10241000F0059091F1050895843040F4763030F461
:102420006F3020F4672F0E94CD11089590E080E076
:102430000895CF92DF92FF920F931F93CF93DF9374
:102440006C010091690680918403082BC7E0D0E0FD
:1024500010E0FC2EC8010C2E02C0959587950A94B9
:10246000E2F780FD0CC02197A0F7F12C8F2DDF91B2
:10247000CF911F910F91FF90DF90CF900895B601FB
:102480008C2F0E94FC110E94240E019761F3EECF65
:10249000CF93DF93EC010E941912BE010E94FC1140
:1024A0000E94240EDF91CF910895FC0180819181DB
:1024B0000E94481292959F70963091F058F4925F66
:1024C0009F70923058F4803F19F030F4883E30F419
:1024D00081E008959A5FF4CF843FD1F380E00895BE
:1024E000883EB0F3813FD1F7F3CF83E290E00E94C2
:1024F000FA318C3289F484E290E00E94FA31823C15
:1025000059F485E290E00E94FA3191E08E3B09F0A7
:1025100090E0892F8170089580E0FCCFCF9384E014
:1025200090E00E94FA31C82F82E290E00E94FA31D6
:10253000982F8C2FCF910895EF92FF920F931F93B6
:10254000CF93DF93062F10E00E541A4FF8019081BD
:10255000992321F1E82EEE0CF0E96F9FE0011124A0
:10256000CE5FDB4F84E2F82EF092EE03EFEEF3E065
:10257000DE018D91819383E0EF3FF807D1F724E6E8
:1025800030E041E150E06EEE73E08E2D0E94BF30EE
:10259000E0E1FE0E6096F4EBFF12E6CFF801108248
:1025A000CDB7DEB7E6E00C941C3160E084E70E9412
:1025B0009C1261E086E70E949C1262E085E70E941F
:1025C0009C120895EEEEF3E06083418324E630E050
:1025D00042E050E0BF01880F0E94BF300895EF92A3
:1025E000FF920F931F93CF93DF93E82E062F10E0F7
:1025F00005511A4FF8018081882381F0F2E16F9F25
:10260000E0011124CB54DA4FF12C49916F2D8E2D1E
:102610000E94E212F39482E1F812F7CFF8011082DF
:10262000CDB7DEB7E6E00C941C31CF93DF93C82F13
:102630004BE06DEF0E94E21240E06AE08C2F0E94B6
:10264000E2128FE39CE90197F1F700C0000040E03F
:1026500060E08C2F0E94E21240E061E08C2F0E942B
:10266000E21240E066E08C2F0E94E21240E06DEF43
:102670008C2F0E94E212D0E040E06D2F8C2F0E9440
:10268000E212DF5FD231C1F740E06D2F8C2F0E9444
:10269000E212DF5FD432C1F740E06D2F8C2F0E9431
:1026A000E212DF5FD43BC1F74BE06DEF8C2F0E944D
:1026B000E21241E06AE08C2F0E94E21240E06DEFEE
:1026C0008C2F0E94E212DF91CF910895A4E0B0E038
:1026D000ECE6F3E10C940131F62E042F122F86352F
:1026E000910570F5880F991F880F991FBC016259D9
:1026F0007A4F44E050E0CE0101960E94C4318981B6
:102700008370EA81282F30E040E9849FC0011124C2
:102710008E5F9B4FE80FF92FF11DB497F082EB818C
:10272000E80FF92FF11DB4970083EC81E80FF92F22
:10273000F11DB49710832E543A4F81E0F901808344
:102740002496E5E00C941D31FF920F931F93CF93D5
:10275000DF93182F062FF42ED0E0C0E02F2D402F4E
:10276000612FCE010E9466132196C635D105B1F7BF
:10277000CDB7DEB7E5E00C941D31A4E0B0E0E3ECAA
:10278000F3E10C94F8300E941C3084E70E9415138A
:1027900086E70E94151385E70E9415130EE615E0E3
:1027A00052E1752E68E0C62ED12CEE24E394F12C74
:1027B0006624639444E050E0B801CE0101960E9483
:1027C000C4314A8150E0CA0184972B81622F645240
:1027D000770B4B012C81E22FE452FF0B5F01298123
:1027E000237030E0FC0197FD379643E0F595E795BF
:1027F0004A95E1F7729EA001739E500D11244B542F
:102800005A4FE40FF52FF11DB6010E942B31A7019D
:1028100001C0440F8A95EAF78081842B8083F401FC
:1028200097FC379693E0F595E7959A95E1F7729EB8
:10283000C001739E900D11248B549A4FE80FF92F0D
:10284000F11DC401B6010E942B31A70101C0440F44
:102850008A95EAF78081842B8083F501B7FC37964F
:1028600083E0F595E7958A95E1F7729EC001739E26
:10287000900D11248B549A4FE80FF92FF11DC501CB
:10288000B6010E942B31A70101C0440F8A95EAF7D7
:102890008081842B808325513A4FF90160820C5F3F
:1028A0001F4FF6E0063C1F0709F084CF60E084E785
:1028B0000E94EF1261E086E70E94EF1262E085E776
:1028C0000E94EF122496EEE00C941431B0E0A0E0E8
:1028D000ECE6F4E10C94FF308C01FC01EB57FD4F6A
:1028E0008081682349F1D0903906D0913A06C09191
:1028F0003806EC2EF12C0E94B431282FC7018C54DD
:102900009F4F68E671E00E942B318E199F0997FD59
:102910000396959587959595879523706C2F289F9D
:10292000600D11247D2D8D2F0E94130A462F282F14
:10293000672FC8010E940C09CDB7DEB7E7E00C9401
:102940001B31B0E0A0E0E7EAF4E10C94FC30182F72
:1029500080911101811323C09091370693702091CB
:10296000100130E081E09217130609F480E08170D5
:102970008093160180913C0690911501981739F0CB
:102980008093150140E060E080E00E940909123167
:1029900060F4E12FF0E0EF55FD4C0C943F3181E005
:1029A000E6CF80911601811102C0C0E0B0C040E0C6
:1029B00060E080E00E940909F8CFC091140182E133
:1029C000C89FC02D112402E10C0FF02E073510F026
:1029D000F6E5FF2E609138067091390680913A062F
:1029E0000E94130AE62ED72EC82ED0E0CF1528F06D
:1029F000C1E0063508F48BC0D8CFFE01EB57FD4F80
:102A0000808190911501892331F02C2D4E2D6D2D53
:102A1000CE010E940C092196E9CFC091140182E1F8
:102A2000C89FC02D112402E10C0FF02E073510F0C5
:102A3000E6E5FE2EE0903806D0913906D0903A06B1
:102A400060913B06669566956695809133069091F8
:102A500034060E94090A0E94BA09805887FD8195B0
:102A6000880F382F2D2D329F312D1124832F6E2D5D
:102A70007D2F0E94130AE62ED72EC82ED0E0CF1548
:102A800008F0B6CFFE01EB57FD4F80819091150104
:102A9000892331F02C2D4E2D6D2DCE010E940C0975
:102AA0002196EDCF8DE899E00E94E40B04C087E009
:102AB00099E00E94510CC82F2AC08EEF98E0F9CF00
:102AC00085EF98E0F6CF87EE98E0EECFC091140145
:102AD00082E1C89FC02D112472E1F72EFC0EEF2C6D
:102AE00086E58F1510F466E5E62E60913B06669547
:102AF00080913306909134060E94090AD82ED0E0C6
:102B0000CE15E8F0C1E025E52F1508F44ECF8091F1
:102B100014018F5F80931401C1110CC082E0809377
:102B2000120180911601811105C0111103C083E0CB
:102B300080931201CDB7DEB7EAE00C941831FE01A4
:102B4000EB57FD4F808190911501892311F1CE0142
:102B5000880F991F81589E4FFC01E55AFF4F208135
:102B60002152330B865A9F4FFC0140814C55550B27
:102B7000609138067091390680913A060D2D0E94B9
:102B8000A9090E94130A462F282F672FCE010E9401
:102B90000C092196B5CF89E799E086CFC091140141
:102BA00082E1C89FC02D112442E1F42EFC0ECF2CEF
:102BB00036E53F1510F436E5C32E60913B06669569
:102BC000669580913306909134060E94090AD82EAA
:102BD00080E48D0D0E94BA0990E8B92EB80E8D2DB3
:102BE0000E94BA0920E8A22EA80ED0E0CC1530F041
:102BF000C1E0E5E5EF1508F08ACFD7CEFE01EB572F
:102C0000FD4F8081909115018923A1F060913806D4
:102C10007091390680913A06ED2C0C2F2A2D4B2D00
:102C20000E940F090E94130A462F282F672FCE01FA
:102C30000E940C092196DACFC0911601C1111EC065
:102C400060913B0620E1620F08F46FEF809133063C
:102C5000909134060E94090A6AE070E00E94E03018
:102C6000892B09F0A2CE0E94B43166E570E00E9483
:102C70002B31609115010E94661449CFC091140157
:102C800082E1C89FC02D112402E10C0F802F07356F
:102C900008F086E5D0E0E82EF12CCE15DF050CF02B
:102CA000A7CE60911501CE010E9466142196F5CF42
:102CB00080EE98E00E94710BFECE8AED98E0FACF8C
:102CC00080913D0621E0382F321B08F430E0832F3D
:102CD00061EC78E00E94A70AEECE80913D0621E0EB
:102CE000382F321B08F430E0832F66E878E0F2CF0B
:102CF00080913D0621E0382F321B08F430E0832F0D
:102D00006EE678E0E7CF68E578E080E0E3CF46E084
:102D100050E06CE170E087E396E00E940832109288
:102D2000ED0308958F929F92AF92BF92CF92DF9260
:102D3000EF92FF921F93CF93DF938091E8039091DE
:102D4000E903A091EA03B091EB032FB7F8948090C8
:102D5000FB059090FC05A090FD05B090FE052FBFEF
:102D600075016401C81AD90AEA0AFB0A2FB7F89458
:102D70004091FB055091FC056091FD057091FE05A9
:102D80002FBF4093E8035093E9036093EA037093E5
:102D9000EB031091BF03EFEBF3E0C12FD0E00197FD
:102DA000AF4FBF4F88199909AA09BB091D1327C046
:102DB000C093BF038091EC03C0E0811108C08091F3
:102DC0003706C82FC37019F0C82FC695C6958091D5
:102DD00012018130F1F1882329F1823009F44AC0CF
:102DE000833009F452C0DF91CF911F91FF90EF9093
:102DF000DF90CF90BF90AF909F908F900895218DDE
:102E0000328D4901B12CA12C88159905AA05BB0565
:102E100020F4C150DF5F3296C9CF2C0D3D1D328F9B
:102E2000218FF8CF1092140140933306509334064B
:102E3000609335067093360689E2EFEBF3E0ADE37D
:102E4000B6E001900D928A95E1F781E0809312013E
:102E5000CACF8C2F0E94A114CC2329F20E9498077C
:102E600081FFC1CF2FEF4FEF6FEF8CE290E00E9418
:102E70000C09B9CFC09311018091370683708093FC
:102E800010010E94D51283E0E1CF8091ED03811102
:102E90000E948716409133065091340660913506A2
:102EA000709136062FB7F8948091FB059091FC0540
:102EB000A091FD05B091FE052FBF841B950BA60BBD
:102EC000B70B4097A105B10508F48DCF1092120100
:102ED0008ACFE7E3F6E085E1808380911701909146
:102EE0001801A091190181839283A3838FE78483C2
:102EF0008FEF85830E948716089590E080E00E94FE
:102F00000232883E9E4F19F40E947512089580E0A7
:102F1000089568EE7EEF90E080E00E94363260E037
:102F200082E090E00E94183260E083E090E00E942E
:102F300018321092840360E084E090E00E9418321E
:102F400064E082E290E00E94183260E085E090E068
:102F50000E94183260E086E090E00E9418326FEF25
:102F600087E090E00E94183240E050E0BA0188E02B
:102F700090E00E942A3260E08DE090E00E941832DA
:102F800040E050E0BA0188E190E00E942A3260E01F
:102F900087E190E00E94183240E050E0BA018CE1F5
:102FA00090E00E942A3270E060E080E290E00E94AF
:102FB000363240E050E0BA0188E190E00E942A32C7
:102FC00080E00E94A4110E94BD1140E050E0BA01CF
:102FD0008FE090E00E942A3240E050E0BA0183E1A5
:102FE00090E00E942A3208951F920F920FB60F921E
:102FF00011242F933F934F935F936F937F938F93FE
:103000009F93AF93BF93EF93FF938091E10082FF73
:1030100009C08091E20082FF05C08091E1008B7FB2
:103020008093E1008091DA0080FF24C08091D80075
:1030300080FF20C08091DA008E7F8093DA0080913B
:10304000D90080FF9DC080E189BD82E189BD09B4BE
:1030500000FEFDCF81E0809332068091040681114D
:1030600009C00E945D050E9450068091E2008460C4
:103070008093E2008091E10080FF17C08091E20020
:1030800080FF13C08091E2008E7F8093E2008091E8
:10309000E20080618093E2008091D800806280939A
:1030A000D80019BC85E0809332068091E10084FF4E
:1030B0002BC08091E20084FF27C080E189BD82E1BE
:1030C00089BD89B5982F917080FFFBCF8091D80082
:1030D0008F7D8093D8008091E1008F7E8093E10006
:1030E0008091E2008F7E8093E2008091E200816017
:1030F0008093E20080912906882309F447C084E088
:1031000080933206809132068091E10083FF27C0D0
:103110008091E20083FF23C08091E100877F80934C
:10312000E10082E080933206109229068091E1004E
:103130008E7F8093E1008091E2008E7F8093E20099
:103140008091E20080618093E20042E060E080E0F4
:103150000E941E068091F00088608093F000FF912D
:10316000EF91BF91AF919F918F917F916F915F91FF
:103170004F913F912F910F900FBE0F901F90189578
:1031800019BC109232061092040674CF8091E300AD
:1031900087FD93E090933206B5CF78941F921FB6C7
:1031A0001F9211248F939F93AF93BF938091FB0540
:1031B0009091FC05A091FD05B091FE050196A11D21
:1031C000B11D8093FB059093FC05A093FD05B09382
:1031D000FE05BF91AF919F918F911F901FBE1F90D1
:1031E00018959C014FB7F8948091FB059091FC05D0
:1031F000A091FD05B091FE054FBF821B930B089572
:103200002FB7F8948091FB059091FC05A091FD05E6
:10321000B091FE052FBF08950E9400199C01909166
:10322000BB038091BC03982B21F03093B80320930B
:10323000B7039091BD038091BE03982B21F030938A
:10324000B6032093B503E091F605F091F7053097AA
:1032500049F082E08093B9030480F581E02D89EB89
:1032600093E009950895ACE0B0E0E9E3F9E10C944E
:10327000FA308E010F5F1F4F8CE0F80111928A9592
:10328000E9F793E5E92E91E0F92E6801AA24A394C9
:10329000B12CF70181917F018F3F09F446C0F8946A
:1032A000E82FE295EF70F0E021A18F70A50102C038
:1032B000440F551F8A95E2F7CA01922F982B91A3CC
:1032C00092A18095892382A3789400C0E9E5F1E07A
:1032D00021E030E0912C812C41914F3F09F489C0CD
:1032E000A42FA295AF70B0E090968C9190E04F70B3
:1032F00002C0959587954A95E2F780FD7AC0C9018D
:10330000882A992A220F331F51E0E836F50721F762
:10331000F701319780818F3F11F00E94CA0D80EA3A
:103320008A95F1F7F60191828082F2E0CF0ED11CEE
:1033300049E5E41641E0F40609F0ABCF4CE050E07B
:10334000B80188E893E00E94CD31FF24F394009700
:1033500009F4F12C892B09F44FC08CE0F801A8E89E
:10336000B3E001900D928A95E1F781E080938703A5
:103370000E940019909386038093850380918503B2
:10338000909186030E94F1180397D0F180918803F1
:10339000909189039093A7038093A60380918A0359
:1033A00090918B039093A9038093A80380918C0341
:1033B00090918D039093AB038093AA0380918E0329
:1033C00090918F039093AD038093AC038091900311
:1033D000909191039093AF038093AE0380919203F9
:1033E000909193039093B1038093B003109287035D
:1033F00007C090E080E084CF809187038111BECF29
:103400008F2D2C96ECE00C941631809180039091D6
:103410007F03892B8093DE0280918303882329F127
:103420000E9400192091810330918203821B930B2B
:103430008838934110F00E94AC0F8091DE02909189
:103440008303892B8093DE02809113018823E1F1AD
:103450008091FF0587FF38C08EE1E0EEF2E090E05A
:103460008150A0F591110E94AC0F40E250E06FE551
:1034700073E08EED92E00E94CD31892B21F180E244
:10348000EEEDF2E0AFE5B3E001900D928A95E1F741
:10349000E091F605F091F7053097A9F080911301BE
:1034A000882359F08091FF0587FF07C08091DE02D5
:1034B0008093DF0286E08093DE020280F381E02DBC
:1034C0008EED92E00995089586E0C7CF21912223E1
:1034D00039F29F5FC5CF90E080E00E94820790E0C4
:1034E00080E00E946C0710927F030E94051A86E01C
:1034F000E9EBF3E0DF011D928A95E9F71092B3033F
:103500001092B2031092B4030E940C190895809394
:1035100069060E946B1A089580916906982F96702B
:10352000963021F488600E94871A0895877FFBCF28
:1035300021E030E001C0220F8A95EAF720958091C2
:10354000690682230E94871A089590915E038095F0
:10355000892380935E03282F277091F4282F082E4B
:10356000000C330B9217130659F09091000692FF4E
:1035700007C08595859585950E94981A0E94BE0F73
:103580000895CF93C0910006C2FB992790F9981730
:1035900091F080FBC2F9C09300066091FF0584E0C2
:1035A00090E00E9418326C2F82E290E00E94183264
:1035B00082E00E94A51ACF91089521E030E001C079
:1035C000220F8A95EAF780916906822B0E94871A5A
:1035D0000895809384030E946B1A089510928003CB
:1035E00080911301E0EEF2E0882361F08091FF0505
:1035F00087FF08C08EE1DF011D928A95E9F70E94DE
:103600006B1A089586E0F7CFAAE2B0E0EAE0FBE1AA
:103610000C9403318AE296E02091F100DC012D93B5
:10362000CD01B6E082339B07B9F780912B0683303A
:1036300009F472C0B8F4813009F449C0823009F449
:10364000B3C08091E80083FF96C280912A069091D2
:103650002B069A3008F08FC2E92FF0E0ED54FD4CB4
:103660000C943F318A3009F48EC08B3009F471C05C
:10367000893039F780912A06813219F780912E0618
:1036800090912F06009711F00297D9F68091E800EB
:10369000877F8093E8008091E80082FF38C0909196
:1036A000F3008091F200029731F48091F1008130B3
:1036B00011F0863021F48091F1008093060680910C
:1036C000E8008B778093E8000E94FF05BACF8091D5
:1036D0002A06813A09F0B5CF8091E800877F809370
:1036E000E80080912E0690912F06892B61F460E20C
:1036F00087E096E070E00E94AB068091E8008B774F
:103700008093E8009ECF60E090E080E0F3CF80916E
:1037100032068111C0CF95CF80912A06813A09F0F7
:1037200090CF80912E0690912F06892B09F089CF9A
:103730008091E800877F8093E8008091E80080FF17
:10374000FCCF809113018093F1008091E8008E7787
:10375000B9CF80912A06813209F073CF80912E066D
:1037600090912F06892B09F06CCF8091E800877F1C
:103770008093E8000E94FF0580912C06809313013E
:103780000E94EE1A5ECF80912A06813209F059CF4D
:103790008091E800877F8093E8000E94FF05809178
:1037A0002D06809305064DCF80912A06813A09F0B7
:1037B00048CF8091E800877F8093E8008091E800FF
:1037C00080FFFCCF80910506BECF803899F082380B
:1037D00009F0D1C180912E068F70873008F0CBC1DF
:1037E0008093E9008091EB0085FB882780F9109297
:1037F000E90006C080912706909128069111826009
:103800009091E800977F9093E8008093F1001092E8
:10381000F1008091E8008E77AAC1882309F498C14D
:10382000823009F0A8C180912C0681119BC1809142
:103830002E068F702FEF280F263008F09CC1809342
:10384000E9002091EB0020FF8DC1933031F480918D
:10385000EB0080628093EB0085C19091EB0090615A
:103860009093EB0021E030E001C0220F8A95EAF747
:103870002093EA001092EA008091EB008860EACF82
:10388000811179C110912C061F778091E300807817
:10389000812B8093E3008091E800877F8093E8008C
:1038A0000E94FF058091E80080FFFCCF8091E3003B
:1038B00080688093E30082E0111183E080933206F8
:1038C0005AC18058823008F056C120912C063091A0
:1038D0002D062C3DE3E03E07A1F583E08A838AE2D2
:1038E00089834FB7F894DE01139620E03EE051E261
:1038F000E32FF0E050935700E49120FF03C0E295DE
:10390000EF703F5FEF708E2F90E0EA30C0F0C79607
:103910008D939D932F5F243159F74FBF8091E8001D
:10392000877F8093E8006AE270E0CE0101960E94F2
:10393000AB068091E8008B778093E8001CC1C096AD
:10394000E7CF80912E0690912F06432F55274330C5
:10395000510509F44AC078F54130510509F485C094
:103960008BE590E0E6E9F9E04230510509F003C14A
:103970002091E800277F2093E800209130063091C5
:1039800031068217930708F49C0140E021153105A8
:1039900009F070C041116EC08091E80082FDC9CF6E
:1039A00080913206882329F2853019F28091E8004F
:1039B00083FFF2CFBECF4132510509F447C04232F6
:1039C000510509F0D8C08330910508F0D4C0FC013E
:1039D000EE0FFF1FED58FE4F0190F081E02D805952
:1039E0009E4FDC018C9190E01DC0332721303105C2
:1039F000E9F02115310579F022303105F9F0233055
:103A0000310509F0B8C0E3E0FAE0E4918E2F90E0D0
:103A1000E3E0FAE007C0E1E4FAE0E4918E2F90E001
:103A2000E1E4FAE0009709F4A6C0A2CFE1E3FAE0EE
:103A3000E4918E2F90E0E1E3FAE0F4CFE1E2FAE0E6
:103A4000E4918E2F90E0E1E2FAE0ECCF8330910533
:103A500008F091C0880F991FFC01E758FE4F0190B4
:103A6000F081E02D89E090E083CF82E190E0E1EF0A
:103A7000F9E07ECF80913206882309F45ACF853051
:103A800009F457CF8091E80083FD53CF8091E8007F
:103A900082FD82CF8091E80080FF78CF9091F30083
:103AA0008091F2002115310519F08830910550F010
:103AB00041E0089709F040E08091E8008E7780931C
:103AC000E80064CF44914093F100319621503109D0
:103AD0000196E8CF803809F04EC08091E800877FDA
:103AE0008093E800809129068093F10092CE8111A5
:103AF00042C010912C061230F0F58091E800877FCB
:103B00008093E800109329060E94FF05112311F00D
:103B100084E005C08091E30087FDFACF81E08093C7
:103B2000320642E061EC81E00E941E0642E261EC56
:103B300084E00E941E0642E261EC82E00E941E06C2
:103B400042E260EC83E00E941E068091320613C0C0
:103B500080912C06813079F481E0933009F080E087
:103B6000809328061092E9008091E800877F809377
:103B7000E8000E94FF058091E80083FF0AC0809161
:103B8000E800877F8093E8008091EB00806280935B
:103B9000EB00AA96E3E00C941F311F920F920FB630
:103BA0000F9211242F933F934F935F936F937F93C3
:103BB0008F939F93AF93BF93CF93DF93EF93FF9335
:103BC000D091E900DF708091EC00C82FC17080FDBA
:103BD000C0E81092E9008091F000877F8093F000A8
:103BE00078940E94041B1092E9008091F000886094
:103BF0008093F000CD2BCF70C093E900FF91EF913F
:103C0000DF91CF91BF91AF919F918F917F916F91F4
:103C10005F914F913F912F910F900FBE0F901F908A
:103C200018950E94EE1A2FEF84E39CE0215080400B
:103C30009040E1F700C0000088E19CE00FB6F894E6
:103C4000A895809360000FBE90936000FFCF8823FB
:103C500041F0809590917F03892380937F030E9498
:103C6000051A0895882339F090917F03982B90933B
:103C70007F030E94051A0895882321F00E94B70F40
:103C80000E94051A0895882339F090918003982B9B
:103C9000909380030E94051A0895882391F19CEF68
:103CA000980F913A40F4682F8EED92E00E940D0734
:103CB0000E94051A089590E2980F983050F487708A
:103CC00091E001C0990F8A95EAF7892F0E94B70FFA
:103CD000EFCF9BE5980F933028F490E080E00E94AE
:103CE0008207089598E5980F973128F490E080E0D6
:103CF0000E946C070895803F20F00E949B0C0E9458
:103D00000C190895CF93C82F8823D1F18CEF8C0F15
:103D1000813AC0F580911301882311F18091FF054C
:103D200087FF1EC0EC2FE695E695E695F0E0E2529F
:103D3000FD4F828190E04C2F477021E030E002C0BF
:103D4000220F331F4A95E2F782239323892B89F0B0
:103D50006C2F8EED92E00E940D070E94051A09C09B
:103D6000E0EEF2E08191C81799F382E0E63EF807B1
:103D7000C9F76C2F8EED92E00E9437070E94051A5A
:103D8000CF91089580E28C0F883068F4C77021E0ED
:103D900030E001C0220FCA95EAF780918003822BA0
:103DA00080938003EBCFEBE5EC0FE33040F4F0E0E1
:103DB000EE5DFE4F808190E00E948207E1CFE8E552
:103DC000EC0FE73150F4F0E0EE0FFF1FEB5DFE4F1C
:103DD000808191810E946C07D3CFC03F88F28C2FE5
:103DE0000E94600D0E940C19CBCF1F93CF93DF93DD
:103DF000182FD0E0C0E0893311F4C0E5D0E0812F66
:103E00000E94821E209739F4812F0E944D1EDF915F
:103E1000CF911F9108958FE99FE00197F1F700C0BE
:103E200000002197EFCF0F931F93CF93DF93C62FFF
:103E3000D42F022FFC0182818823A9F060936806A9
:103E40000E9400199093670680936606C77081E010
:103E500001C0880FCA95EAF70E94431EDF91CF91F7
:103E60001F910F91089580916806681332C0809168
:103E70006606909167060E94F118883C910548F506
:103E800010E21D0FCD17B9F080E28C0F883040F49E
:103E9000C77081E001C0880FCA95EAF70E943C1EF6
:103EA000183048F481E09D2F977001C0880F9A95D3
:103EB000EAF70E94431E802F0E94F51E183070F60C
:103EC000D77081E001C0880FDA95EAF70E943C1EA6
:103ED000C5CFC77081E001C0880FCA95EAF7F6CF59
:103EE000B0E0A0E0E6E7FFE10C94FC30EC018AE0F2
:103EF000A82E2881222309F48FC02130C9F5998189
:103F00008A81913021F422960E94F51E05C09230DC
:103F100029F422960E94821E2196EBCF933021F441
:103F200022960E944D1EF8CF943011F02196F4CFC6
:103F3000229630E020E0AE014F5F5F4F8053990B37
:103F40008A30910550F02150310930F38FE99FE01C
:103F50000197F1F700C00000F6CFA29EB001A39E2A
:103F6000700D11249C01260F371F8981EA01E3CFD0
:103F7000E22FF0E0E650FE4FB490822F86958695B2
:103F8000869590E0FC01E651FE4FE4902770F12CFD
:103F9000022E02C0F594E7940A94E2F731E0E3229E
:103FA000FF24FC01E652FE4FC490D12C022E02C029
:103FB000D594C7940A94E2F731E0C322DD24FC01D2
:103FC000E653FE4F049110E002C0159507952A951F
:103FD000E2F701701127E114F10419F081EE0E945B
:103FE000821EC114D10419F086EE0E94821E8B2D10
:103FF0000E94F51EC114D10419F086EE0E944D1ED8
:10400000E114F10419F081EE0E944D1E0115110515
:1040100009F482CF8CE278CFCDB7DEB7EAE00C941A
:1040200018319091000692FF10C098E0899F90018E
:104030001124622B60935E030E94DD1A0E94001916
:1040400090935D0380935C0308950E94DD1A0895A8
:10405000A7E1B0E0EEE2F0E20C9403314B8B5C8B15
:104060006D8B7E8B8F8B611110927F031A8A198A58
:1040700085E0FE017396DE011D9601900D928A95F2
:10408000E1F78091000682FF1CC00E940019209178
:104090005C0330915D03821B930B8838934120F0C1
:1040A00080915E0382FF78C00E94001920918103F5
:1040B00030918203821B930B8838934110F00E9449
:1040C000AC0F86E0FE013D96DE01179601900D9241
:1040D0008A95E1F7CE0107960E949E27811112C0B2
:1040E00086E0FE013796DE01119601900D928A95C9
:1040F000E1F78A859B85892B29F088859F81892313
:104100008F3F81F516E080915B0390912A0389131C
:1041100017C06796E3E00C941F3196E0929FD001A0
:10412000939FB00D1124A55DBC4FFE013196019007
:104130000D929A95E1F780932A030E94C50FE2CF72
:10414000819FC0011124855D9C4F0E949E2788237A
:1041500001F380915B0390E001968770992780932B
:104160005B03D1CF20912A0330E0C901019687700B
:10417000992740915B034817190679F60E94EE1AB9
:1041800010922A0310925B0386E0E4E2F3E0DF0181
:104190001D928A95E9F7B6CF82E00E94A51A84CFD6
:1041A000A5E0B0E0E6EDF0E20C9402318C019093D2
:1041B000F1058093F005011580E21807C0F4802F07
:1041C0000E944D1EC8010E943A109801205E3109DC
:1041D0002830310518F00115110531F40E943C1EFC
:1041E0002596E4E00C941E310E94271EF9CF80EF43
:1041F00089838A831B820E9400198160782F9D83A6
:104200008C8349815A816B818D810E942820E8CF5F
:10421000A5E0B0E0EEE0F1E20C9402318C01909365
:10422000F1058093F005011580E21807C0F4C8017C
:104230000E943A109801205E31092830310518F0AB
:104240000115110549F40E94431E802F0E94821E11
:104250002596E4E00C941E310E94321EF6CF80EFCA
:1042600089838A8381E08B830E9400198160782F83
:104270009D838C8349815A816B818D810E94282086
:10428000E7CFA5E0B0E0E7E4F1E20C94FA306C018E
:10429000FC0183819481892B31F080819181892374
:1042A0008F3F09F058C52596ECE00C9416310E941A
:1042B0001912182F682F89819A810E940310698131
:1042C0007A81812F0E94FC118C01F6018281882362
:1042D00009F436C5980122513F452031310508F0D7
:1042E00008C58FEF93E00E94FA318111A5C00251F9
:1042F00057EFA52E52E0B52E011133C019821A8254
:104300001B821C82EE24EA9445013FEF831A930A34
:10431000C5010E94FA3189831A82882309F48CC06E
:10432000813009F07EC085010E5F1F4FC4010E94DD
:10433000FA31F82E8A83882309F47EC0C8010E94CE
:10434000FA31982E8FEF8F0D8330D0F40F5F1F4F0F
:104350009B82992021F0CE0101960E94701F580186
:10436000D3CFA114F4E0BF0609F466C0C5010E94D2
:10437000FA31811101C001502FEFA21AB20ABCCF4D
:104380008BEF8F0D833040F5C50103969B828C0126
:10439000992029F385010C5F1F4F0E94FA318C830D
:1043A0008823E9F2AB80BC8041E0A4164FEFB4064D
:1043B00010F0BA2CAA2456E0F51651F087E0F81652
:1043C00019F0C5010E940821C5010E94D020C7CF65
:1043D000C5010E940821C3CF94E0F912C0CF850126
:1043E0000C5F1F4FC50103960E94FA31992021F1FD
:1043F000882311F18150990BE89E9001E99E300DC0
:104400001124E92DE150FF0BCF01820F931F01977B
:1044100008F4A5CFEFE9FFE03197F1F700C0000005
:10442000F6CFCE0101960E94701F840198CF81E0E3
:104430000E94DD1A0E948C1A80915E03877009F435
:1044400032CFF6018281882309F42DCF80910006B6
:1044500082FF29CF82E00E94A51A25CF81E00E9429
:10446000981AE8CF82E0E4CF053FECE51E0709F497
:1044700061C008F45BC0063F2CE5120709F45EC07A
:10448000882309F479C41092680603303DE51307C8
:1044900008F05BC00A3F4CE5140730F4C8018250B5
:1044A0009C45449708F05BC00E948E1290930006D2
:1044B0008093FF0501319CE5190709F42DC108F02F
:1044C000A7C00930FCE51F0709F414C108F072C049
:1044D00005303CE5130709F405C108F057C0033067
:1044E0005CE5150709F4F4C008F0F8C08091FF05F9
:1044F000816002309CE5190709F4EDC06091FF0569
:104500001091000684E090E00E941832612F82E250
:1045100090E00E9418320E94EE1A8ECF27E245EEFC
:1045200065EE0AC426E241EE60EE06C427E245EEDF
:1045300064EE02C426E241EE62EEFEC327E245EEDF
:1045400066EEFAC328E241E0EBCF01365DE51507E0
:1045500009F4AACF053A8DE5180709F4A5CF06316D
:10456000ECE51E0709F077C4809180038A7A91E018
:1045700009F490E09093FE0269E2811165E38EED0B
:1045800092E00E9437070E94051A56CF8091FF05DE
:1045900080620730ECE51E0709F49DC08091FF059D
:1045A00080610830FCE51F0708F495C08091FF0585
:1045B000806491C08091FF058B7F0D302CE5120740
:1045C00009F489C0A0F48091FF058E7F0B304CE583
:1045D000140709F480C08091FF058C600C305CE505
:1045E000150708F478C08091FF058D7F74C00F30E7
:1045F0008CE5180709F48CC08091FF05877F003196
:104600009CE5190708F467C08091FF058F7D63C0A2
:104610000D3FECE51E0709F477C058F505312CE590
:10462000120709F483C098F48091FF05837F03315A
:104630004CE5140709F44FC008F472C00E94EE1A4A
:104640009091FF05892F97FB87F9805844C00B3F55
:104650008CE5180709F44AC008F052C080910006A2
:1046600081600A3FECE51E0709F048CF8093000601
:1046700045CF0130FDE51F0709F464C0C0F4809107
:1046800000068C7F0F3F3CE5130781F38091000605
:10469000836001154DE5140748F380910006982FBB
:1046A000909591708E7F892B90FB81F9DFCF013639
:1046B0005DE5150709F44CC0053A8DE5180709F4C6
:1046C0004EC002309DE5190709F018CF60E03BC0ED
:1046D0008091FF0582608093FF0510CF8091FF05D8
:1046E0008460F9CF8091FF058860F5CF8091000646
:1046F0008260BCCF0E94EE1A8091FF058068EBCFEC
:10470000809100068E7FB2CF809100068D7FAECF64
:104710008091FF058F7EDFCF8091FF058F7BDBCF00
:104720000E94EE1A8091FF058F77D5CF8091FF050B
:1047300082FB992790F921E0922790FB82F990FB68
:1047400083F9C9CF61E08EE090E00E941832D6CEA6
:104750009091FF05892F8F7E94FF8061BCCF90914F
:10476000FF05892F8E7F90FF8160B5CF8091FE027B
:1047700069E2811165E38EED92E00E940D0703CF9F
:1047800041E458E06CE478E00E94A50755CE4CE483
:1047900058E061E478E0F8CF42E158E06DE178E07C
:1047A000F3CF4DE158E062E178E0EECF46EF57E01D
:1047B00064E078E0E9CF44E058E066EF77E0E4CFEA
:1047C00048EE57E06AED77E0DFCF4BEA57E069EB60
:1047D00077E0DACF49EB57E06BEA77E0D5CF61E0DD
:1047E00081E00E94280828CE61E085E0FACF0E948F
:1047F000EE1AFFEF24E33CE0F15020403040E1F7B7
:1048000000C000000E9400118091000682FB8827F2
:1048100080F991E089270E94C11AF6018281008106
:104820001181882309F445C0C8010E941912F82E8D
:10483000682FC8010E940310B8018F2D0E94FC113F
:104840000E94240E8C01882EF601E280B580B2947D
:104850003FE0B32280915E038770C1F0AE2CEE2062
:10486000B1F0812F807F803421F080E2800F88308A
:1048700068F08091000682FF09C082E00E94A51ABC
:1048800080915E038770AA24A3948111A12C912E9C
:1048900092942FE09222FBE0F91508F476C0E92DFE
:1048A000F0E0E354FD4C0C943F3181E0B4CF80E064
:1048B000B2CFC8010E94CF0FF82EBECF212F2F708C
:1048C000F22E107F19F0F29490EFF922EE20B9F059
:1048D000FF2069F080E2800F883010F0811009C05D
:1048E00080918003F82AF09280030E94051A802F9D
:1048F0004AC080917F03F82AF0927F03F6CF802F81
:104900000E944D1EFF2009F440C0005E083010F0E8
:10491000811004C08F2D0E94B70F06C0F0948091C3
:104920007F03F822F0927F030E94051A2EC0312FD8
:104930003F70F32E107F103219F0F29480EFF822BE
:10494000882089F041E0841609F491C0EE2009F432
:104950009AC0BB2009F467C0F601858180FFC7CFEC
:104960008F70858360C08091000682FD35C0EE2087
:1049700069F1FF2039F080918003F82AF0928003DA
:104980000E94051A80E00E94821E292D2850330BB8
:104990002430310510F40E949807AA2009F483CC32
:1049A00080915E0380FD7FCCF6011282859585950E
:1049B00085950E94DD1AC6010E94412180915E0307
:1049C0008595859585950E94981A6DCC80E00E940A
:1049D0004D1EFF20D1F29ECFEE2049F1B11004C050
:1049E000809183038F2920C051E0B51210C082FF4F
:1049F000CCCF80918303F82AF81639F20E9400196F
:104A00009093820380938103F0928303BECF85E06D
:104A1000B812E6CF0E94AC0F9091FF028F2D892B28
:104A200089138093FF028F2D0E94431EAECFB110D9
:104A300003C00E94AC0F12C091E0B91213C0809164
:104A400080038F2109F4A1CF0E94AC0F9091FF0247
:104A50008F2D8095892389138093FF028F2D0E94CB
:104A60003C1E93CFE5E0BE1609F48FCFE2CFEE20D7
:104A700029F0F5E0FB1508F488CFD5CF24E02B15FD
:104A800008F483CFEBCFBB2049F3F9E38F1209C0C1
:104A90002FEF37EE43E0215030404040E1F700C0B7
:104AA0000000802F0E944D1E70CF812F8695869525
:104AB000837061F0813009F068CFC8019370E11014
:104AC00002C090E080E00E946C075FCFC801937045
:104AD000E11002C090E080E00E94820756CF802F54
:104AE000EE2029F00E94600D0E940C194ECF0E940A
:104AF0009B0CFACF812F837089F5E11046CF402FB0
:104B0000429546954770440F440F802F8F70042EB6
:104B100001C0880F0A94EAF7202F207104FF07C014
:104B20002FE030E001C0220F4A95EAF72095169554
:104B300016951370123069F050F4309184031130DF
:104B400029F0822B83230E94E91A1FCF832B822B0B
:104B5000FACF282B809184038227F5CF8695EE200B
:104B600011F0812F8170882309F40FCF402F4295D7
:104B700046954770440F440F802F8F70042E01C05C
:104B8000880F0A94EAF7202F207104FF07C02FE056
:104B900030E001C0220F4A95EAF720951695169548
:104BA0001370123069F050F430916906113029F019
:104BB000822B83230E94871AE8CE832B822BFACF85
:104BC000282B809169068227F5CF1F70EE2029F0EF
:104BD000812F0E94DD1A802F27CF802F0E943C1E3C
:104BE000812F0E94981AD1CE802F52EF8516B1F1F5
:104BF000581570F090EF8916D1F0E1EF8E1691F014
:104C0000EE2009F466C0B11072CE812F8F712AC0D8
:104C1000F3EF8F1651F124EF8212F2CF809100064C
:104C200082FD2FC0812F8F71EE20D9F21BC0EE20A4
:104C300081F034E03B1508F4A8CE1F7181E090E0CC
:104C4000012E01C0880F0A94EAF79091690689271E
:104C5000B1CF45E04B1508F498CEEFCF812F8F717F
:104C6000E110BFCF0E94DD1A90CE80E0EE2009F463
:104C7000A1CF1F7181E0012E01C0880F0A94EAF7CD
:104C800099CFEE20C9F080915E038770843041F4A3
:104C90000E94BE0F812F8F710E94981AA12C75CE91
:104CA00054E05B15D8F31F71812F0E94DD1A63E079
:104CB000812F0E941120F2CF84E08B1530F40E94E6
:104CC000BE0F64E0812F8F71F4CF81E00E94A51A9E
:104CD000E5CFBB2059F0893309F0E3CE9FEFE7EE33
:104CE000F3E09150E040F040E1F7D9CE812F8F7191
:104CF00078CF0031FFE51F0709F499CB01312FE58B
:104D0000120709F4AFCB033F2CE5120709F40ACCD4
:104D100008F0AACB083D4CE5140709F4FFCB093D88
:104D20005CE5150709F40ECC073D9CE5190709F071
:104D3000A7CB26E241EE61EEC6010E94131F7CCB99
:104D400000313FE5130709F489CB01314FE5140722
:104D5000D1F682E084CB85E0DE01119601900D92C0
:104D60008A95E1F7F601228189819A8121119FCAF2
:104D70000E94CF0F182FA3CA0631FCE51F0709F4C4
:104D8000F5CC8091800382720A3C2CE5120709F46D
:104D900017CDB0F5053C4CE5140709F4FDCCD0F473
:104DA000033C9CE5190709F4EBCC08F0F0CC023C7D
:104DB000FCE51F0709F031CD8091370691E0892786
:104DC00080933706109212018091ED0381608093E9
:104DD000ED0332CB073C2CE5120709F4E7CC08F4CD
:104DE000E0CC083C4CE5140709F4E5CC093C5CE553
:104DF000150709F012CD4AED57E068EE77E0C4CC14
:104E00000F3C9CE5190709F4EFCCA0F40C3CFCE541
:104E10001F0709F4DFCC08F4D8CC0D3C3CE51307A0
:104E200009F4DDCC61E082E00E3C4CE5140709F4A6
:104E3000D8CCF3CC063D5CE5150740F4013D8CE58C
:104E4000180708F0F9CA61E088E0CBCC0D351007EF
:104E500009F4F2CAE2CC0A35EDE51E0709F425CDC6
:104E600068F401152CE5120709F4C1CC0E3D1C4570
:104E700009F0D3CC0E9489170E94111E0C354DE514
:104E8000140709F4C1CC08F412CD073A1D45A1F36B
:104E9000C4CC1F93CF93DF9380912903807F09F0C7
:104EA00049C080912603882309F444C080915B03A4
:104EB000D0912A036091240370912503A0912703C8
:104EC000B0912803C62FC72316E0D81799F190E0B8
:104ED000109711F0CF3F19F401968770F6CF189F05
:104EE0009001199F300D1124F901E55DFC4F4181BE
:104EF0004713F2CF40814613EFCF42814111ECCFEF
:104F0000438154814A1B5B0B483C510528F7809133
:104F100029038F70806180932903F901E05DFC4FC4
:104F200080818F708061808384E293E00E944121C0
:104F30000E94C50FDF91CF911F910895A1E1B0E0CC
:104F4000E4EAF7E20C94FC308C0185E0F801DE0124
:104F50001D9601900D928A95E1F7F801E28084E2B6
:104F6000A82E83E0B82E6091270370912803611565
:104F7000710509F426C19091240340912503892FDE
:104F800084238F3F09F41DC120813181C380D480E7
:104F9000F0902603F601E61BF70BFF2009F4DCC0B6
:104FA00080912903582F507FE83CF10508F09FC0FD
:104FB00051116BC0FE2C431314C0921312C0E110A8
:104FC00010C08F70806180932903C5010E94412128
:104FD00080912903F80185838F2D6196EAE00C9476
:104FE0001831C114D10429F0822F83238F3F09F097
:104FF00003C180E0F82FF170DF2E80FF3CC080916C
:105000005B0340912A0356E0841315C02D873E8729
:105010008D859E850E944812292F22952F7022305F
:10502000F0F0243018F59F70F1F0F8019581907F31
:10503000D1F4D12C1EC090E0589FF001599FF00D83
:105040001124E55DFC4F6181361306C06081261393
:1050500003C06281E6120FC001968770D5CF9F70A2
:1050600011F0882331F3805E883018F3C8010E9464
:105070004121FD2CB1CFEE2009F4AECF8091290360
:10508000816080932903F12CA7CF431306C09213AC
:1050900004C0F801EE2009F479C0C8010E9455123D
:1050A000882309F1EE20F9F080912903803270F015
:1050B000209124033091250338872F831986DB86BE
:1050C000CA868C87CE0107960E94412186E0F801AE
:1050D000A4E2B3E001900D928A95E1F70E9449277E
:1050E000FF24F39479CFC8010E944121F9CF5111D7
:1050F0000AC084E293E00E94412186E0F50111920A
:105100008A95E9F7C0CF43130FC092130DC0E11089
:105110000BC0F8018583C8010E94412186E0F5019A
:1051200011928A95E9F758CFC8010E945512882339
:10513000D1F2EE20C1F280912903803238F2209121
:105140002403309125033A8329831B82DD82CC829C
:105150008E83CE010196B8CFE83CF105F8F6FE2C1F
:10516000EE2009F243131FC092131DC08091290342
:1051700080FD10C0982F907F69F0F8018583903FE3
:1051800031F0982F907F905F8F70892B8583C801B5
:105190000E94412186E0F801A4E2B3E001900D9263
:1051A0008A95E1F719CFC8010E94551281118ECF5F
:1051B00080912903816080932903C8010E944121C5
:1051C0000BCFEE2009F48FCFC8010E945512F82EA4
:1051D000882309F488CF86E0F801A4E2B3E00190C7
:1051E0000D928A95E1F780912403909125030E9406
:1051F00048120E944927F0CE81E08E25FBCE1F92F7
:105200001FB61F9211248F939F93AF93BF938091EA
:10521000FA05811113C08091FB059091FC05A091C6
:10522000FD05B091FE054196A11DB11D8093FB05C2
:105230009093FC05A093FD05B093FE05BF91AF913F
:105240009F918F911F901FBE1F901895CDB7DEB70D
:10525000E4970FB6F894DEBF0FBECDBF85B7806868
:1052600085BF85B7806885BF84B7877F84BF0FB649
:10527000F894A895809160008861809360001092F6
:1052800060000FBE80E890E00FB6F8948093610054
:10529000909361000FBE88EC9DE09093DD028093B7
:1052A000DC020E945D050E9450068091E20084604D
:1052B0008093E2007894809132068823A1F01091C7
:1052C000E9001F709091EC00892F817090FD80E8BB
:1052D000182B1092E9008091E80083FD0E94041BC6
:1052E0001F701093E90082E084BD93E095BD9AEFB2
:1052F00097BD80936E000E947512811102C00E94BA
:10530000BD1103E511E0D8018D918D018F3F11F0A2
:105310000E94CA0DB1E009351B07A9F709E511E0A4
:1053200038E6E32E31E0F32EF80181918F018F3FB3
:1053300011F00E94CA0DE016F106B1F78CE0E6EA22
:10534000F3E0DF01282F1D922A95E9F7E8E8F3E062
:10535000DF011D928A95E9F70E947D17811102C035
:105360000E94891782E090E00E94FA3180939403B2
:105370000E948E12909300068093FF050E943319BD
:10538000EFEBFDE53197F1F700C000000E94331903
:105390008091A60380FF08C06FEF7FEF90E080E070
:1053A0000E9436320E94001183E090E00E94FA31A0
:1053B0000E94E91A0E94BD1310923D068FEF9FEFE5
:1053C00090935706809356069093590680935806FB
:1053D00090935B0680935A0690935D0680935C06DB
:1053E00090935F0680935E069093610680936006BB
:1053F000909363068093620690936506809364069B
:105400001092BF039093D9038093D8039093DB034A
:105410008093DA039093DD038093DC039093DF03A2
:105420008093DE039093E1038093E0039093E30382
:105430008093E2039093E5038093E4039093E70362
:105440008093E6030E947D17811104C00E94891792
:105450000E94691746E050E06CE170E087E396E057
:105460000E94EA311092ED03809137068C7F11F48F
:105470000E94691784E091E09093F7058093F60508
:10548000332433948091320623E0F22E00E112E1BE
:10549000853009F4F5C00E943319882359F08FB77D
:1054A000F8944091FB055091FC056091FD057091C9
:1054B000FE058FBF96EAE92E93E0F92EE5E9F3E0C9
:1054C000D70110E000E0602FCD90DD902191319167
:1054D0002C153D0509F41CC2912CAA24A394B12CCF
:1054E0002C253D25A9014A215B21452B09F40AC23F
:1054F00099A66AA7CA20DB2081E0C114D10409F46F
:1055000080E08BA70E9400198160782F9DA78CA74F
:1055100049A55AA56BA58DA50E942820F801EE0F7C
:10552000FF1FEB56FC4F80819181A826B926B182DE
:10553000A082CD2871F08FE0809FF001819FF00D57
:105540001124E158FE4FE90DF11D80818F3F09F0D4
:10555000A3C0B12C0B2D10E08091BF03800F912FC1
:10556000911D09976CF188E090E06C01C01AD10A96
:10557000B80160547C4FA60180EC93E00E94DA31C0
:10558000B80168537C4FA60188EC93E00E94DA31A1
:10559000A601440F551FB801660F771F68527C4F54
:1055A00088ED93E00E94DA31B80160537C4FA60188
:1055B00080ED93E00E94DA3188E08B198093BF037D
:1055C0008091BF0390E0A22DB0E09D01220F331F18
:1055D00027523E4FAA0FBB1FBD0166527E4F74C0BB
:1055E00080913206843009F43AC00E94921680916C
:1055F000EC0381110DC00E94A11410921101809141
:1056000037068370809310010E94D512F092120128
:10561000F1E0F093EC031092FA0528E130E040E469
:105620000FB6F894A895209360000FBE40936000D9
:1056300083B7817F846083BF83B7816083BF7894A1
:10564000889583B78E7F83BF0FB6F894A895809115
:105650006000886180936000109260000FBE8091AE
:105660002806882369F00E943319E6EAF3E0819165
:105670009191892B09F0B8C483E0E23BF807B9F7B0
:1056800080913206853009F4ABCF0E94EE1A0E9459
:1056900098071092EC03FFCE282EBB24B3945ACF68
:1056A00090E0FC01E154FC4FD9015C915183DB0196
:1056B0005C915187218A880F991FFC01E154FC4FAE
:1056C000128E118E91E0842F41E0480F9B1540F31C
:1056D0008093BF030E94921686E0E9EBF3E08E010F
:1056E0000F5F1F4FD80101900D928A95E1F710923C
:1056F000BB031092BC031092BD031092BE038B81BA
:105700009C81892B09F44AC08091B7039091B8031A
:105710000E94F1189C019091B303992309F487C466
:1057200025313105D8F19F3F19F09F5F9093B30366
:10573000DB80DD2059F00E94400D9FEF1D140CF41A
:1057400091E0899F802D11248093BB03DC80DD20B4
:1057500059F00E94400D9FEF1D140CF491E0899FB9
:10576000802D11248093BC033091BB033323B1F00F
:105770002091BC03222391F045EB3403C001112496
:10578000992309F4DCC09093BB0345EB24039001FB
:105790001124332309F4D6C03093BC038D819E813C
:1057A000892B09F44AC08091B5039091B6030E94F9
:1057B000F1189C019091B203992309F433C4213567
:1057C0003105D8F19F3F19F09F5F9093B203DD80C0
:1057D000DD2059F00E941E0D9FEF1D140CF491E086
:1057E000899F802D11248093BD03DE80DD2059F038
:1057F0000E941E0D9FEF1D140CF491E0899F802DD7
:1058000011248093BE033091BD033323B1F0209166
:10581000BE03222391F045EB3403C00111249923E8
:1058200009F493C09093BD0345EB24039001112428
:10583000332309F48DC03093BE0346E050E0B80135
:1058400089EB93E00E94CD31892B61F48091BB03F9
:105850009091BC03892B9091BD03892B9091BE033D
:10586000892B11F00E940C1986E0F801A9EBB3E036
:1058700001900D928A95E1F70E9498079091A103FB
:1058800089138093A10380913206843009F0FACD08
:1058900083E08093E9008091E80082FFF3CD80915E
:1058A000E80090E085FF0AC00E947C0530E2A32E4C
:1058B000B12C6801882309F458C091E08091E80078
:1058C0008B778093E800992309F4DCCDC090F20532
:1058D000D090F3058981C114D10409F454C08E3FDE
:1058E00009F0E5C08A81833020F08550833008F0CC
:1058F000DEC0EA81EE3008F0DAC0F0E0E753FD4C9C
:105900000C943F319394AA0CBB1C4FE09412EACD47
:105910000F5F1F4F0630110509F0D5CD8FEF8EA711
:105920008FA718AA0E9400198160782F9AAB89ABC3
:105930004EA55FA568A98AA90E942820CBCE3092E7
:10594000BB0323CF3092BC0329CF3092BD036CCF71
:105950003092BE0372CF8091F100D6018D936D011C
:10596000B1E0AB1AB10809F4A8CF8091E80085FD39
:10597000F2CF8091E8008B778093E8000E947C054D
:10598000882399F39ACF8B3009F440C258F58530BB
:1059900009F4B7C0D0F4823009F46FC030F481301C
:1059A00009F467C08FEF898382C0833009F49AC0FD
:1059B0008430C1F74C816B818A810E94CD11982778
:1059C000892798279E838D8372C0873009F4A7C0EA
:1059D00008F4A2C0883009F4DFC0893019F70E94AA
:1059E000871665C0803109F462C1B8F58D3009F4BD
:1059F00032C108F42DC18E3009F42FC18F3091F6D9
:105A00008091EE059091EF05892B09F450C0EC8050
:105A1000F12CFDE1EF16F10408F049C0CA80DB80EB
:105A2000DC24CD24DC245801E00EF11EC60189508F
:105A30009D4FAE14BF04D9F129E0C21621E0D20671
:105A400028F4D50114966C910E941832BFEFAB1A5E
:105A5000BB0AEFEFCE1ADE0AE9CF823109F42CC17E
:105A600008F428C1833109F450C18E3F09F09ACF60
:105A700040CF1A8289E08B831AC08A81823009F470
:105A8000C9C28330C1F0813009F08CCF2FB7F894B0
:105A90006091FB057091FC058091FD059091FE05DC
:105AA0002FBF0E9445316B837C838D839E83C80109
:105AB0000E94D705E7CC8091EE059091EF05892BE8
:105AC000B1F3F801D7018C9111969C91B2E0EB0EE5
:105AD000F11C92838383329622EBE21623E0F206D6
:105AE00089F7E5CF8A81823009F05CCF6B817C81B8
:105AF0008D819E810E94453186E290E00E9418329D
:105B0000D6CF2D813E813227232732274C816B81CE
:105B10008A810E943411CBCF0E945A11C8CF8A814A
:105B2000813429F64B815C8180913706982F9370E0
:105B30004115510589F49111109212018C7F8093C7
:105B400037068D8180933B068E8120E048856F81EA
:105B500090E00E94C707ABCF911102C010921201D2
:105B60008C7F81608093370626E234E06EE674E035
:105B7000F901329685919491F901A591B4914A1752
:105B80005B0731F02C5F3F4F6217730789F780E0A6
:105B900060E00E942808D5CF8A81813459F0823490
:105BA00009F436C0803409F082CF3B821C8288EC35
:105BB0008D837DCF80913706982F9370C1F08695A5
:105BC000869590E026E234E06EE674E0F9013296C4
:105BD000A591B491F90145915491E42F452F8A176D
:105BE0009B0739F02C5F3F4F6217730779F7E0E0AE
:105BF00040E0EB834C8380913B068D838091380697
:105C00008E83809139068F8380913A0688874FCFA3
:105C1000EB80FC804EE150E06FEF70E0CE01039628
:105C20000E94E33186E294E0DE0113962EE1FC014E
:105C300045915491E416F50628F4223018F04D935E
:105C40005D932250049634E08E36930781F72FCF70
:105C500080E18A832CCF3A820DCFEC80F12C4DE18C
:105C6000E416F10408F023CFCA80DB80DC24CD24C5
:105C7000DC245801E00EF11EC60189509D4FEA1444
:105C8000FB0409F414CFA9E0CA16A1E0DA0658F41F
:105C90000E94FA31F5018483BFEFCB1ADB0AEFEFE4
:105CA000AE1ABE0AE9CFD50114961C92F5CF0E9418
:105CB0002411FDCE84E0CDCFEC80F12CFDE1EF1678
:105CC000F10408F0F4CECA80DB80DC24CD24DC248F
:105CD0005801E00EF11EC6018796EA14FB0409F490
:105CE000E6CE20EDC21622E0D20660F40E94FA3120
:105CF000D50114968C93FFEFCF1ADF0A2FEFA21A6B
:105D0000B20AE9CFF5011482F6CFCC80D12C3DE167
:105D1000C316D10408F0CBCEEA80FB80FE24EF242A
:105D2000FE2440EDE41642E0F40608F0C0CE80ED1B
:105D300092E08E199F098C159D0508F4B8CE3701A5
:105D400087E2680E711C8091EE059091EF052701A6
:105D50004C0C5D1C892BB9F5570191E0A922BB249D
:105D6000E0FE0DC0C70186960E94FA319D81892709
:105D70009827892781159C4511F48FEF8D83460163
:105D800040FE1AC0B1E08B1A9108E5E0F0E0EC0F9C
:105D9000FD1FE80DF91DFCABEBABC3018C0D9D1D88
:105DA0000E94FA31ABA9BCA99C9181159C4521F4B4
:105DB0008FEFEBA9FCA98083F801EA0DFB1D2FEF03
:105DC000A814B90410F068011BC094818581811565
:105DD0009C4511F42483258342E0A40EB11C329625
:105DE000EFCFA0EDEA16A2E0FA0620F4F6016481F6
:105DF0000E941832FFEFCF1ADF0A2FEFE21AF20AE1
:105E0000C70187964E145F0461F751CE8091EE056D
:105E10009091EF05892B09F44ACEC8010E94D7055D
:105E20003FEF41EE84E0315040408040E1F700C058
:105E30000000B8CA88E0EAE1F1E0DE019196019045
:105E40000D928A95E1F780E2D8011D928A95E9F7D3
:105E500085E0898388E0FE01B196DE011596019008
:105E60000D928A95E1F73D8622CE8CEA89833A82AB
:105E70001B821C821CCE8C81682F70E0762F6627D7
:105E80008B81860F972F911D092E000CAA0BBB0B3F
:105E900025E0880F991FAA1FBB1F2A95D1F7AC01D7
:105EA000BD01405E5F4F6F4F7F4F481759076A072C
:105EB0007B0708F4FCCD8C3AE1E09E07A105B10513
:105EC00008F0F5CD4D3AF1E05F076105710520F06E
:105ED0004CEA51E060E070E0481B590BBC01665889
:105EE0007D4FC8010E94C431E2CD4AE150E06FEF1E
:105EF00070E0CE0107960E94E3318091EE05898320
:105F0000CA821B821C8283E08D838DE08E83CFCD7D
:105F100081E090E09093F3058093F20582E390E0B6
:105F20009093A5038093A4030E9400199093A30368
:105F30008093A203BCCDCD2889F1D090A603E09038
:105F4000AC03F090AD038091A2039091A3030E9453
:105F5000F1188536910558F1F5FAEE24E0F8EE20B7
:105F600031F1D0FE24C00E9400199093A3038093C6
:105F7000A2038091A4039091A50301979093A50398
:105F80008093A403892B51F41092F3051092F2052B
:105F900081E090E09093EF058093EE058091EE050F
:105FA00089838091F2058A838091A40364CD82E382
:105FB00090E09093A5038093A403F0CF1092EF0597
:105FC0001092EE0574CD40E250E06FEF70E0C80132
:105FD0000E94E3316CCD8B81811169CD80E2D801C3
:105FE0001D928A95E9F763CD09BD19BD09B400FE7C
:105FF000FDCF8091D8008F7D8093D8008091E00004
:1060000082608093E0008091E00081FDFCCF0E94DF
:10601000EE1A36CB86E290E00E94FA311B821C8297
:106020001D8274CF2B30310508F0CECB06CC2B303F
:10603000310508F07ACBB2CB1092B9008CE0809396
:10604000B8000895B0E0A0E0E8E2F0E30C94FB3083
:10605000B82EEB010E9400196C01EE24E394F12CA0
:10606000C431D10560F025E0E22EF12CCF3FDC07F2
:1060700031F0CE0164E170E00E94E0307B0184EAFF
:10608000A82E94E8992E1092BC00A092BC000E9409
:1060900000198C018091BC0087FF0DC08091B90070
:1060A000887F883001F18091B900887F8031D9F0F4
:1060B0000FEF1FEF09C00E940019801B910B8E1576
:1060C0009F0540F30EEF1FEFCF3FDC07E1F2C60163
:1060D0000E94F1188C179D07B0F2C801CDB7DEB74A
:1060E000EBE00C941731B092BB009092BC000E9480
:1060F00000198C018091BC0087FF0AC08091B90013
:10610000887F883111F0803499F610E000E0E5CF07
:106110000E940019801B910B8E159F0558F3D2CF5A
:106120000F931F93CF93DF93EB018093BB0084E821
:106130008093BC000E9400198C018091BC0087FFF5
:1061400011C02091B900287F81E090E0283211F43D
:1061500090E080E0919581959109DF91CF911F9119
:106160000F910895CF3FDC0741F30E940019801B77
:10617000910B8C179D0708F38EEF9FEFEECFB0E0E9
:10618000A0E0E5ECF0E30C94FE306B018A017901AC
:10619000B9010E942230E6010C0D1D1DC017D10768
:1061A00011F097FF08C024E92093BC00CDB7DEB7FB
:1061B000E8E00C941A31B70189910E949030EECF3B
:1061C000AA1BBB1B51E107C0AA1FBB1FA617B7071D
:1061D00010F0A61BB70B881F991F5A95A9F7809539
:1061E0009095BC01CD0108952F923F924F925F92FE
:1061F0006F927F928F929F92AF92BF92CF92DF92D7
:10620000EF92FF920F931F93CF93DF93CDB7DEB73B
:10621000CA1BDB0B0FB6F894DEBF0FBECDBF0994CF
:106220002A88398848885F846E847D848C849B8426
:10623000AA84B984C884DF80EE80FD800C811B8134
:10624000AA81B981CE0FD11D0FB6F894DEBF0FBE63
:10625000CDBFED01089597FB072E16F4009407D0EB
:1062600077FD09D00E94E03007FC05D03EF4909500
:1062700081959F4F0895709561957F4F0895EE0F1A
:10628000FF1F0590F491E02D09946927962769274F
:106290007827872778270895CF92DF92EF92FF9291
:1062A000CF93DF93CDB7DEB72A970FB6F894DEBF52
:1062B0000FBECDBF89879A87A985BA852D913D915B
:1062C0004D915C9129833A834B835C83232B242B50
:1062D000252B41F424E239ED4BE557E029833A833D
:1062E0004B835C8369817A818B819C812DE133EFC3
:1062F00041E050E00E943C3269017A01A7EAB1E432
:106300009B01AC010E945B3269837A838B839C83FF
:10631000ACEEB4EFA70196010E9469329B01AC017B
:1063200089819A81AB81BC81820F931FA41FB51F05
:10633000B7FF03C00197A109B048E985FA858083BA
:106340009183A283B3839F772A960FB6F894DEBF1A
:106350000FBECDBFDF91CF91FF90EF90DF90CF9038
:1063600008950E944C31089580E091E00E944C31E4
:106370000895B0E0A0E08093000190930101A09304
:106380000201B09303010895FB01DC0102C00590F6
:106390000D9241505040D8F70895FB01DC0104C034
:1063A0008D910190801921F441505040C8F7881B0D
:1063B000990B0895FB01DC0102C001900D92415040
:1063C0005040D8F70895DC0101C06D934150504012
:1063D000E0F70895DC01CB01FC01F999FECF06C07E
:1063E000F2BDE1BDF89A319600B40D924150504093
:1063F000B8F70895F999FECF92BD81BDF89A992713
:1064000080B50895A8E1B0E042E050E00C94EC3192
:10641000DC01A40FB51F4150504048F0CB01840F60
:10642000951F2E910E94193241505040D0F7089587
:10643000262FF999FECF92BD81BDF89A019700B43D
:10644000021639F01FBA20BD0FB6F894FA9AF99ADD
:106450000FBE08950396272F0E9419320E9418320A
:10646000252F0E941932242F0C9419320196272FC0
:106470000E9419320C941832052E97FB1EF40094DA
:106480000E94533257FD07D00E946E3207FC03D0A2
:106490004EF40C94533250954095309521953F4FD2
:1064A0004F4F5F4F089590958095709561957F4F00
:1064B0008F4F9F4F08950E949032A59F900DB49FDB
:1064C000900DA49F800D911D11240895B7FF0C9489
:1064D0005B320E945B32821B930B0895A1E21A2E5D
:1064E000AA1BBB1BFD010DC0AA1FBB1FEE1FFF1F78
:1064F000A217B307E407F50720F0A21BB30BE40BC8
:10650000F50B661F771F881F991F1A9469F760950E
:106510007095809590959B01AC01BD01CF010895C8
:10652000A29FB001B39FC001A39F700D811D1124D4
:10653000911DB29F700D811D1124911D0895F89435
:10654000FFCFD114DD140D15521557155D156015CB
:1065500063156615CB15CE151C1658165D166016FC
:106560006D1678168316E51B0D1CBB1D0D1CBB1D7F
:10657000401C611CBB1D6A1D771D5E245E24972490
:10658000972455256F25C524C5247A25E525F425AE
:10659000F4251A2F352F3B2F572D572D752F882F68
:0E65A0009B2FDE2FE32F572D572D572DEB2F5E
:1065AE00010000000A07C0109F109A1095100907ED
:1065BE00FFFF030100FF0000FFC8A05204CE2345D9
:1065CE00716D818283E200E900EA00B500B600B782
:1065DE0000CD008301CC008A019201940121022397
:1065EE000224022502260227022A02B300B4006FFB
:1065FE00007000F7F6F5F4F1F03031323337929344
:10660E009594969734353666003131295A1B750AA2
:10661E004022BC8A016801AC00A809C109E1090049
:10662E000102030405060708090A0B0C0D0E0F10D4
:10663E0011121314FF15161718191A1B1C1D1E1FE5
:10664E00202122232425262728292A2B2C2D2E2FC4
:10665E00303132333435363738393A3B3C3D3E3FB4
:10666E00404142434445464748FF494A4BFF4C4D43
:10667E004E4FFF505152535455000010001E002B28
:10668E00003800480055006300700080008D009AAD
:10669E0000A700BE00D800000D100D200C310E42D8
:1066AE0010521466147610860E960CA70DB80DC5F2
:1066BE000DD80D001A0F1A1F172F183F1C4E1EE073
:1066CE001A691E781C88189817A81AB81AC51AD2F3
:1066DE001A00250F251E212D233C254B285C2B6CE3
:1066EE00287C258A239921A825B825CB25E02500CD
:1066FE00300E301D2C2B2E393048325C3570327EE8
:10670E00308D2E9B2CA930B830D230003A0E3A2262
:10671E003A3D3D534064407A3D953AAA3AB83AC55F
:10672E003AD23AE03A0404040404040404040404CF
:10673E00040404040404040404040404040404040B
:10674E0004040404040404040404040404040404FB
:10675E0004040404040404040404040404040404EB
:10676E0004040404040404040404040404010404DE
:0C677E00040404040404040401010100EC
:00000001FF
